:100000000C947E0B0C94DE400C943E410C949B0BA4
:100010000C949B0B0C949B0B0C9448410C949B0BE5
:100020000C949B0B0C9452410C949B0B0C949B0BCB
:100030000C949B0B0C949B0B0C949B0B0C949B0BA8
:100040000C94B8410C949B0B0C949B0B0C949B0B45
:100050000C94DE410C9406420C9435420C949B0B9C
:100060000C949B0B0C949B0B0C949B0B0C949B0B78
:100070000C949B0B0C949B0B0C949B0B312E3233EA
:100080002E30300017151515151517001212121203
:10009000121212001711111714141700171111174B
:1000A0001111170015151517111111001714141738
:1000B0001111170017141417151517000000000070
:1000C0000000000084008C0094009C00A400AC00A0
:1000D000B400BC004845414400474554202F00521D
:1000E00045424F4F540D0A0052455345540D0A00E6
:1000F0004A4A59004750530054532D4E5450303102
:100100005F585858585858006E74702E6A73742E81
:100110006D666565642E61642E6A70003030302E25
:100120003030302E3030302E303030003030302E05
:100130003030302E3030302E303030003030302EF5
:100140003030302E3030302E3030300008011C017D
:100150002C013C01F40614073407540730313233C4
:1001600034353637383941424344454600485454C3
:10017000502F312E312032303020485454500D0A47
:10018000436F6E6E656374696F6E3A20636C6F7354
:10019000650D0A436F6E74656E742D547970653AFF
:1001A00020746578742F68746D6C0D0A4361636800
:1001B000652D436F6E74726F6C3A206E6F2D6361A4
:1001C0006368650D0A436F6E74656E742D4C616EC5
:1001D00067756167653A20656E0D0A0D0A0048541F
:1001E00054502F312E3120323030204F4B0D0A43E6
:1001F0006F6E6E656374696F6E3A20636C6F7365C2
:100200000D0A436F6E74656E742D547970653A20D3
:10021000746578742F68746D6C0D0A43616368654A
:100220002D436F6E74726F6C3A206E6F2D63616335
:1002300068650D0A436F6E74656E742D4C616E6750
:10024000756167653A20656E0D0A0D0A3C21444FC1
:1002500043545950452048544D4C205055424C4928
:100260004320222D2F2F5733432F2F44544420480F
:10027000544D4C20342E3031205472616E736974A9
:10028000696F6E616C2F2F454E2220226874747046
:100290003A2F2F7777772E77332E6F72672F54523E
:1002A0002F68746D6C342F6C6F6F73652E6474647B
:1002B000223E3C48544D4C3E3C484541443E3C5413
:1002C00049544C453E54532D4E54502D534552568F
:1002D00045522053455455503C2F5449544C453EAB
:1002E0003C2F484541443E3C424F445920424743FD
:1002F0004F4C4F523D2223464646464646464622EE
:100300003E3C43454E5445523E3C423E00223E3C1C
:100310002F464F524D3E3C42523E3C464F4E54209B
:10032000434F4C4F523D22475245454E223E564187
:100330004C55452053415645443C2F464F4E543E64
:100340003C42523E00223E3C42523E3C42523E3CE7
:10035000494E50555420545950453D225355424D15
:100360004954222056414C55453D224150504C594C
:10037000223E3C2F464F524D3E004950004E4D000C
:10038000475700444E004243007A037D03800383B5
:100390000386032000240028002C00C0006401A86C
:1003A000C000FFFFFF0101A8C00101A8C0FF01A814
:1003B000C049502041444452455353005355424E86
:1003C0004554204D41534B00474154455741590036
:1003D000444E5320534552564552004144445245E1
:1003E000535300B103BC03C803D003DB034E3100F9
:1003F0004E32004E33004E3400ED03F003F303F6AB
:1004000003534552564552310053455256455232D8
:1004100000534552564552330053455256455234C7
:10042000000104090411041904400060008000A0C8
:100430000000504F574552204F4E004558544552EA
:100440004E414C2052455345540042524F574E2086
:100450004F55542052455345540057415443484446
:100460004F472054494D455220524553455400456D
:100470004E4332384A36302052454345495645208E
:100480004552524F5200415250205245515545530A
:10049000542054494D454F5554204552524F520017
:1004A00049434D50205041434B4554204348454318
:1004B0004B2053554D204552524F5200544350202B
:1004C0005041434B455420434845434B2053554DE1
:1004D000204552524F5200554450205041434B4505
:1004E0005420434845434B2053554D204552524FCD
:1004F000520049434D50204D455353414745004418
:100500004843502052454345495645204E414B28CB
:1005100052455452592900444843502052454E45B3
:1005200057414C20535441544500444843502052B5
:100530004542494E44205354415445004448435099
:100540002045585049524544205354415445004495
:100550004843502052454345495645205041434B5E
:100560004554204552524F52004E4254205245436A
:1005700045495645204552524F52004E425420465E
:100580004F524D4154204552524F52004E4254203A
:100590005041434B4554204552524F52004E425415
:1005A0002054494D45204F555428534552564552E5
:1005B0003129004E42542054494D45204F5554286E
:1005C0005345525645523229004E42542054494D0B
:1005D00045204F5554285345525645523329004E15
:1005E00042542054494D45204F55542853455256A6
:1005F0004552342900444E532054494D45204F550F
:100600005428534552564552312900444E532054E4
:10061000494D45204F55542853455256455232298D
:1006200000444E532054494D45204F5554285345BE
:1006300052564552332900444E532054494D4520CB
:100640004F5554285345525645523429004E545064
:1006500020554E53594E43524F4E495A4544004E31
:1006600054502054494D45204F5554285345525617
:1006700045523129004E54502054494D45204F5584
:1006800054285345525645523229004E5450205456
:10069000494D45204F55542853455256455233290C
:1006A000004E54502054494D45204F555428534531
:1006B000525645523429004E545020494C4C45471F
:1006C000414C20534552564552205245504C5900FA
:1006D0004E5450204C454150205345434F4E4420EA
:1006E00041444A5553540054494D4520494C4C45CA
:1006F00047414C00475053204E4D454120464F52F4
:100700004D4154204552524F52004E4D45412043D9
:100710004845434B53554D204552524F5200544982
:100720004D452044415441205245434549564520BA
:100730004552524F5200554E53594E432054494D45
:1007400045555000310432043B044A045A046F04F6
:100750008604A004BC04D704F204FF0417052A058C
:100760003C054F0569057B058C059D05B305C9054D
:10077000DF05F5050B06210637064D065F067506F3
:100780008B06A106B706D006E706F4060A071E0781
:1007900036076E772E636769006E732E6367690094
:1007A0006E622E63676900636C2E63676900656C17
:1007B0002E6367690073642E6367690066617669FA
:1007C000636F0092079907A007A707AE07B507BC9C
:1007D00007464958204E4554574F524B20534554D5
:1007E00054494E470054494D4520534552564552B1
:1007F0002053455454494E470054494D45205052CA
:100800004F564944452053455454494E4700544996
:100810004D452042524F414443415354204C4F4791
:10082000004556454E54204C4F47005359535445AC
:100830004D20494E464F4D4154494F4E00D107E59A
:1008400007F9070E0821082B084E54502041444A4E
:100850005553544D454E54204D4F44450042524F40
:100860004144434153542041444A5553544D454E0D
:1008700054204D4F4445004750532041444A55535E
:10088000544D454E54204D4F4445004A4A5920434B
:100890004C4F434B2041444A5553544D454E5420F0
:1008A0004D4F44450049085D0877088B084E4F209E
:1008B000414C41524D2854494D452053594E4352C5
:1008C0004F4E495A4544290054494D4520414C4119
:1008D000524D284E4F542053594E43524F4E495A71
:1008E0004544290054494D4520554E41444A5553ED
:1008F0005445440054494D45204F504552415449B8
:100900004F4E2054494D454F555400465552554E73
:100910004F20525443204D4F444500465552554EAA
:100920004F20475053204D4F444500555443204DD0
:100930004F44452856414C494429005554432050C2
:1009400050534F5554204D4F44452856414C49442F
:100950002900554E49564750532054494D45204E85
:100960004F2056414C4944004E4F2054494D45209C
:10097000494E50555400AD08C808E408F4080B0966
:100980001B092B093B095209680920485454502F70
:10099000003C2F413E3C42523E003F223E003C4242
:1009A000523E3C4120485245463D222E2F00545392
:1009B0002D4E54502D5345525645523C2F423E3CED
:1009C00042523E004243004954424C00223E3C42C7
:1009D000523E3C42523E494E54455256414C285399
:1009E00065632E2030206F72203E3635353334203B
:1009F00049676E6F7265293C42523E3C494E5055E4
:100A00005420545950453D225445585422204E41BB
:100A10004D453D224954424C222053495A453D22DE
:100A20003822204D41584C454E4754483D223522EE
:100A30002056414C55453D22003530223E3C2F5436
:100A4000483E3C54482057494454483D22313530B3
:100A5000223E54494D453C2F54483E3C5448205773
:100A6000494454483D22313530223E414D4F554E88
:100A7000543C2F54483E3C54482057494454483D28
:100A800022313530223E4E4F54453C2F54483E3C97
:100A90002F54523E003C2F54443E3C2F54523E00B3
:100AA0003C2F54443E3C54443E26656D73703B00DD
:100AB0003C2F54443E3C54443E42432041444A551A
:100AC0005354006D732E007365632C006F7665724E
:100AD0002039686F7572732E00444953545249424D
:100AE0005554494F4E002D2D2D2D2D3C2F54443E55
:100AF0003C54443E003C2F54443E3C54443E00266B
:100B0000656D73703B003C2F54443E3C54443E00A2
:100B10003C545220414C49474E3D2243454E54459A
:100B200052223E3C54443E004552525253540043DC
:100B30004C520050473D3100313530223E54494D32
:100B4000453C2F54483E3C54482057494454483D66
:100B500022353030223E4556454E543C2F54483EB7
:100B60003C2F54523E003C2F54443E3C2F54523EA6
:100B70000026656D73703B3C2F54443E3C54443E0C
:100B800026656D73703B002C44415441313A002C72
:100B9000434F44453A0028545950453A002C4E459D
:100BA00058543A002C434E543A00285354533A00B8
:100BB0003C2F54443E3C54443E002D2D2D2D2F2DD2
:100BC0002D2F2D2D202D2D3A2D2D3A2D2D003C543D
:100BD0005220414C49474E3D2243454E54455222F6
:100BE0003E3C54443E003C2F5441424C453E3C4226
:100BF000523E004F5045524154494E472054494DB2
:100C000045004D494E2E00484F555220004649524E
:100C10004D574152452056455253494F4E00454E7F
:100C20004332384A3630205245564953494F4E00D8
:100C30004D414320414444524553530054494D458E
:100C400020535441545553004F5045524154494F3D
:100C50004E204D4F4445004E455442494F53204E7F
:100C6000414D4500444E532053455256455200478E
:100C70004154455741592041444452455353005330
:100C800055424E4554204D41534B0049502041445C
:100C9000445245535300323030223E4954454D3C76
:100CA0002F54483E3C54482057494454483D223331
:100CB0003030223E56414C55453C2F54483E3C2F47
:100CC00054523E003C2F54443E3C2F54523E003C74
:100CD0002F54443E3C54443E003C545220414C4925
:100CE000474E3D2243454E544552223E3C54443EDD
:100CF00000222056414C55453D220022204D4158AE
:100D00004C454E4754483D2200222053495A453D08
:100D100022003C42523E3C494E50555420545950BA
:100D2000453D225445585422204E414D453D220018
:100D3000223E3C42523E003C42523E3C2F43454EF6
:100D40005445523E3C2F424F44593E3C2F48544D4F
:100D50004C3E003C42523E3C4120485245463D22DA
:100D60002E2F223E4D41494E204D454E553C2F41A0
:100D70003E3C42523E003C42523E003F455252529F
:100D80005354223E4552524F52204F46463C2F412B
:100D90003E3C42523E0026656D73703B3C4120480C
:100DA0005245463D22003F434C52223E4C4F472085
:100DB000434C4541523C2F413E003F50473D31227C
:100DC0003E5B325D3C2F413E26656D73703B3C417E
:100DD00020485245463D22003F50473D30223E5B71
:100DE000315D3C2F413E26656D73703B3C41204890
:100DF0005245463D22003C2F5441424C453E3C4228
:100E0000523E3C4120485245463D22003C2F423E46
:100E10003C42523E3C42523E3C5441424C452042B0
:100E20004F524445523D2231223E3C54523E3C54A6
:100E3000482057494454483D220022204D455448FB
:100E40004F443D22474554003C2F423E3C42523ED7
:100E50003C464F524D20414354494F4E3D22005392
:100E6000554E004D4F4E00545545005745440054D3
:100E70004855004652490053415400414955545287
:100E8000475550564E54532D4E54502D534552569F
:100E90004552303100454E4332384A3630205245B3
:100EA000563A00494E495449414C495A494E472EF9
:100EB0002E2E00494E495449414C495A4544004B55
:100EC0004559494E50555420494C4C4547414C00DA
:100ED0004D544B3333333920494E49542E2E2E0076
:100EE00043414C2052454D3A004448435020444928
:100EF0005341424C4544004448435020454E4142F2
:100F00004C4544004E545020525820454E41424CCE
:100F10004544004E54502052582044495341424CBD
:100F200045440042524F414443415354204C4F47A3
:100F3000004F5045524154494E472054494D4500B9
:100F4000475053204D4F4445205245414459004A93
:100F50004A59204D4F444520524541445900465579
:100F600052554E4F20475053204D4F444500554E4B
:100F7000495620475053204D4F444500454E43327B
:100F8000384A363020494E495445525200850E9514
:100F90000EA30EB30EBF0ED00EE00EE90EF70E0438
:100FA0000F130F230F310F400F4F0F5E0F6E0F7C8B
:100FB0000F56657273696F6E00504C454153452062
:100FC000434845434B204B455900504C4541534500
:100FD000205245534554004D41433A004448435044
:100FE000434E543A004E42432052454D3A00574139
:100FF000495420666F722054494D45205258004391
:101000004F4E4E4543542054532D4A4A59303200D6
:10101000434845434B204349524355495400504CA3
:1010200045415345205741495400434845434B20CF
:10103000434F4E4E4543544F5200B10FB90FCA0FA4
:10104000D70FDC0FE50FEE0FFF0F10101E102A1048
:1010500045585049524544200020524542494E448B
:10106000200052454E4557414C2000494E46494EBE
:10107000495459005010591062106B104A535400D3
:101080004B535400434354005554430050535400B1
:10109000484454007C108010841088108C109010EC
:1010A0002020202020202020202020202020202040
:1010B00000504F574552204F4E0045585445524E10
:1010C000414C2052455345540042524F574E204FF9
:1010D0005554205245534554005741544348444FBA
:1010E0004720524553455400454E43205243562015
:1010F0004552524F520041525020524551205449BE
:101100004D454F55540049434D502053554D2045B2
:1011100052524F52005443502053554D2045525285
:101120004F52005544502053554D204552524F5276
:101130000049434D50204D455353414745205243AC
:101140005600444843502052454345495645204E99
:10115000414B00444843502052454E4557414C00B6
:101160004448435020524542494E4400444843506D
:10117000204558504952454400444843502050436C
:1011800054204552524F52004E4254205243562052
:101190004552524F52004E425420464F524D4154F8
:1011A000204552524F52004E4254205041434B452D
:1011B00054204552524F52004E42542054494D45FE
:1011C0004F5554284E6F3129004E42542054494DFA
:1011D000454F5554284E6F3229004E4254205449F1
:1011E0004D454F5554284E6F3329004E42542054DC
:1011F000494D454F5554284E6F342900444E5320D5
:1012000054494D454F5554284E6F312900444E5393
:101210002054494D454F5554284E6F322900444EB5
:10122000532054494D454F5554284E6F332900449F
:101230004E532054494D454F5554284E6F34290084
:101240004E545020554E53594E43524F4E495A45D5
:10125000004E54502054494D454F5554284E6F313F
:1012600029004E54502054494D454F5554284E6F37
:101270003229004E54502054494D454F5554284E64
:101280006F3329004E54502054494D454F55542832
:101290004E6F3429004E545020494C4C4547414C28
:1012A000205245502E004E5450204C454150204174
:1012B000444A5553540054494D4520494C4C4547E8
:1012C000414C0047505320464F524D415420455207
:1012D000524F52004E4D45412043484B53554D20EF
:1012E0004552522E0054494D45204441544120520C
:1012F000435645525200554E53594E432054494D82
:1013000045555000A010B110BA10C910D910E810FE
:10131000F6100611151123113111421153116011EC
:101320006C11791188119611A711B811C911DA1130
:10133000EB11FC110D121E122F12401251126212EB
:10134000731284129512A612B612C312D412E512A9
:10135000F6122D2D2F2D2D202D2D3A2D2D3A2D2D00
:1013600000484F55522020204D494E2E002A2A3A3F
:101370002A2A3A2A2A002D2D3A2D2D3A2D2D0054B5
:10138000494D450D0A00444154450D0A0061646A07
:1013900075737465640076616C69640053545553C9
:1013A0000D0A00444353540D0A002D2D5A444100A8
:1013B00047505A4441002D2D524D43004750524D45
:1013C0004300504645432C475074707300504D54B1
:1013D0004B3030312C3331342C330024504D544BAE
:1013E0003331342C302C312C302C312C302C302C0F
:1013F000302C302C302C302C302C302C302C302C0D
:10140000302C302C302C312C302A32390D0A00246B
:10141000504D544B3331342C302C312C302C312C5A
:10142000302C302C302C302C302C302C302C302CDC
:10143000302C302C302C302C302C302C302A3238C0
:101440000D0A004649582049502041444452455312
:101450005300464958205355424E4554204D415360
:101460004B004649582044464C5420474154455768
:1014700041590046495820444E5320534552564541
:10148000520044484350205553452F554E5553451F
:1014900000424C4F41444341535420414444522E56
:1014A00000424C4F41444341535420494E54564C02
:1014B0000042434153542043414C20524543562E51
:1014C0000054494D45205A4F4E4500475053204E39
:1014D0004F444154412054494D45520047505320F8
:1014E000554E53594E432054494D4552004E4D459B
:1014F000412053454E54454E5345003150505320E2
:10150000494E5055542045444745004E54502052B2
:10151000582054494D454F55540041444A55535461
:1015200020574944544800475053204241554420D5
:1015300052415445005155495420544F204D414982
:101540004E00431452146214731482149114A114A3
:10155000B114C114CB14DC14ED14FB140B151A15C3
:10156000271535154A5354285554432B393A3030F2
:1015700029004B5354285554432B393A3030290015
:10158000434354285554432B383A3030290055549E
:10159000432855544320303A3030290050535428C2
:1015A0005554432D383A3030290048445428555476
:1015B000432D393A303029006415721580158E1587
:1015C0009C15AA15907E0000907E0000807000009F
:1015D00000000000808FFFFF7081FFFF46555255CD
:1015E0004E4F282447507470732900554E49562E8B
:1015F00028244750524D432900554E49562E282441
:1016000047505A44412900DC15EB15F91546414C69
:101610004C204544474500524953452045444745E1
:10162000000D16171644495341424C4500454E41A2
:10163000424C450025162D1644495341424C450065
:10164000454E41424C45284E5450204D4F4445296B
:10165000003816401620313230306270730020326C
:101660003430306270730020343830306270730070
:101670002039363030627073003139323030627068
:1016800073003338343030627073003537363030A1
:101690006270730055165E166716701679168216FC
:1016A0008B1657494454483A202020202073656304
:1016B0000054494D454F55543A20202020206D7349
:1016C00000544F55543A2020202020736563005465
:1016D0004F55543A202020202073656300494E5412
:1016E000455256414C3A202020202073002F31379C
:1016F000002D2D204D454E55202D2D0011241FBEAF
:10170000CFEFD0E1DEBFCDBF12E0A0E0B1E0E8E076
:10171000F8EC02C005900D92AC3BB107D9F71BE085
:10172000ACEBB2E001C01D92A83AB107E1F70E940C
:10173000E80E0C9402640C94000080917C018823D4
:1017400059F480916A0990916B0990938B0B809367
:101750008A0B81E080937C010895A0E2B0E0E3EB86
:10176000FBE00C9497620E94F01982E00E94F94B12
:1017700001C0A895F999FDCF86E090E065E070E0A2
:101780000E94FD6301C0A895F999FDCF8EE090E01D
:1017900060E570E00E94FD6301C0A895F999FDCF56
:1017A0008CE090E06AE070E80E94FD6301C0A895BB
:1017B000F999FDCF80E290E044E651E068EA70ECF0
:1017C0000E94F56301C0A895F999FDCF84E290E0ED
:1017D00040E05FEF6FEF7FEF0E94F56301C0A895D7
:1017E000F999FDCF88E290E041E051E068EA70ECC1
:1017F0000E94F56301C0A895F999FDCF8CE290E0B5
:1018000041E051E068EA70EC0E94F563CE01019678
:1018100068EF70E00E94F06201C0A895F999FDCFD1
:10182000CE01019660E170E040E150E00E94DD638E
:1018300001C0A895F999FDCF8E010F5F1F4FC80118
:1018400068E071E00E94F062C80160E470E040E28C
:1018500050E00E94DD6301C0A895F999FDCF8E018B
:101860000F5F1F4FC8016CE171E00E94F062C80178
:1018700060E670E040E250E00E94DD6301C0A895A0
:10188000F999FDCF8E010F5F1F4FC8016CE271E027
:101890000E94F062C80160E870E040E250E00E94FF
:1018A000DD6301C0A895F999FDCF8E010F5F1F4F31
:1018B000C8016CE371E00E94F062C80160EA70E068
:1018C00040E250E00E94DD6301C0A895F999FDCF88
:1018D00080EC90E04FEF51E068EA70EC0E94F56315
:1018E00001C0A895F999FDCF84EC90E060E070E02C
:1018F0000E94FD6301C0A895F999FDCF86EC90E0A8
:1019000060ED77E00E94FD6301C0A895F999FDCFD5
:1019100088EC90E068E873E10E94FD6301C0A8953F
:10192000F999FDCF8CE390E061E070E00E94FD63E7
:1019300001C0A895F999FDCF8CEC90E060E070E0D3
:101940000E94FD6301C0A895F999FDCF80ED90E05C
:1019500064EB70E00E94FD6301C0A895F999FDCF8A
:1019600082ED90E064E873E00E94FD6301C0A895F9
:10197000F999FDCF8EE390E065EA73EC0E94FD6378
:10198000A096E4E00C94B3620F931F930E94561D3F
:1019900083B180958F70873069F40E94AD0B0E94EF
:1019A000F01983E00E94F94B82E00E94EC4BA8956D
:1019B000FECFA895F999FDCF8EE390E00E94A36336
:1019C000855A934C21F00E94AD0B01C0A895F9995E
:1019D000FDCF86E090E00E94A3639C0101978E5F9B
:1019E0009F4F10F025E030E020930F0401C0A89530
:1019F000F999FDCF8EE090E00E94A3639093E704F5
:101A00008093E60401978E5F9F4F40F080E590E061
:101A10009093E7048093E60401C0A895F999FDCF5F
:101A20008CE090E00E94A3639C019F779093D6077F
:101A30008093D507C90101978E5F9F4F50F084E1D5
:101A40008093D8078CE390E09093D6078093D507D6
:101A500010C037FF0CC080916E0990916F090197FB
:101A600011F084E101C085E18093D80702C0109293
:101A7000D8078091D807882309F040C080E290E021
:101A800044E651E068EA70EC0E94051C6093AD04E6
:101A90007093AE048093AF049093B00484E290E01E
:101AA00040E05FEF6FEF7FEF0E94051C6093B10491
:101AB0007093B2048093B3049093B40488E290E0EE
:101AC00041E051E068EA70EC0E94051C6093B504A7
:101AD0007093B6048093B7049093B8048CE290E0BE
:101AE00041E051E068EA70EC0E94051C60936109D6
:101AF00070936209809363099093640980E190E098
:101B000061E579E048EF50E00E94E21B809103011B
:101B10006AE579E00E94C13B809104016CE579E0BF
:101B20000E94C13B809105016EE579E00E94C13BB6
:101B300080ED90E00E94A3632FEF8F3F920711F496
:101B400084EB90E0909369098093680982ED90E0BE
:101B50000E94A3634FEF8F3F940711F484E893E052
:101B600090936B0980936A0980E490E064EF76E0DB
:101B700048E051E00E94BF1B80E690E064E177E01E
:101B80004CE151E00E94BF1B80E890E064E377E005
:101B90004CE251E00E94BF1B80EA90E064E577E0F0
:101BA0004CE351E00E94BF1B80EC90E04FEF51E00E
:101BB00068EA70EC0E94051C60937A0770937B07BB
:101BC00080937C0790937D0701C0A895F999FDCF7C
:101BD00084EC90E00E94A36390939B0780939A0704
:101BE0008F5F9F4F31F410929B0710929A0701C0AC
:101BF000A895F999FDCF86EC90E00E94A36390939D
:101C000099078093980701978E5F9F4F40F080ED72
:101C100097E0909399078093980701C0A895F99948
:101C2000FDCF88EC90E00E94A3639093A00780937F
:101C30009F078F5F9F4F31F488E893E19093A0074F
:101C400080939F0710916709012F077011F011C051
:101C5000A895F999FDCF8AEC90E00E94A36397FDC7
:101C600008C080FF06C0187F11601093670901C08B
:101C7000A895F999FDCF8CE390E00E94A3634FEF04
:101C80008F3F940711F480E090E00230E1F420915E
:101C90006709277C20936709AC0147705070413079
:101CA000510511F4286004C04230510519F4206137
:101CB0002093670983FF07C0809167098064809340
:101CC000670901C0A895F999FDCF8CEC90E00E94BE
:101CD000A363809375098F3F21F41092750901C0A9
:101CE000A895F999FDCF80917509E82FF0E0EE0FE6
:101CF000FF1FEE0FFF1FEC53FA4E85919591A591B2
:101D0000B4918093770190937801A0937901B09377
:101D10007A011F910F910895EF92FF920F931F93F5
:101D2000E0909A07F0909B0700E010E083E591E0D7
:101D30006DE171E00E94EE3EE61AF70A080B190BFE
:101D4000B701C8011F910F91FF90EF900895EF9296
:101D5000FF920F931F93E0909C07F0909D07002740
:101D6000F7FC0095102F81E491E06DE171E00E9495
:101D7000EE3EE61AF70A080B190BB701C8011F91CE
:101D80000F91FF90EF9008950F931F938C010E9485
:101D9000E03D005110406F717070060F171F1093D7
:101DA0009D0700939C070C33110534F48CE390E0FD
:101DB00090939D0780939C07A1E4B1E0EDE1F1E0F1
:101DC00082E101900D928150E1F71F910F910895EA
:101DD000A4E0B0E0EEEEFEE00C948962F89410927C
:101DE00068001CBA1DBA89E88093640080E885BF4A
:101DF00085BF80BF9FEF92B980E185B918B813E025
:101E00001BB991B980EB84B98FE787B982EC8AB9A5
:101E100088E090E00E949D636093A1077093A20701
:101E20008093A3079093A40789B18073803129F42C
:101E3000119882E08093670905C0803239F41298C6
:101E40001093670989E080937D0103C01098109278
:101E5000670980E18CBD81E08DBD16BC92E094BD28
:101E600083E085BD27EC27BD90936E001092B200F1
:101E70009093B00084E08093B1002093B3009093DE
:101E8000700084B780FF04C081E00E94C24F13C07D
:101E900081FF02C082E007C082FF02C083E003C06E
:101EA00083FF09C084E00E94C24F81E090E09093DC
:101EB0006F0980936E0914BE8CE028E130E00FB604
:101EC000F894A895209360000FBE809360007894EA
:101ED0000E946F1A0E94C40C80E58CBD8091670936
:101EE0008770823011F580910F04882319F484E300
:101EF00095E01FC0813019F48AE992E01AC082305F
:101F000019F48CE491E015C0833089F0843019F421
:101F100082E590E00EC0853019F489E290E009C0B6
:101F2000863059F48BE190E004C0833089F485EA6F
:101F300090E09093C5008093C40082E08093C0003D
:101F400086E08093C20088E98093C1008091C6003A
:101F50005E9A80E190E00E94C21A0E949315882345
:101F600081F484E162EA7AE00E94C2140E94F019CE
:101F700081E10E94F94B88E00E94EC4B1798A895EC
:101F8000FECF0E9469180E94F01980E00E94F94B70
:101F900080E00E94EC4B88E061E04CE750E00E945A
:101FA000211AC090670927E0C2220E94C91A8C0139
:101FB0000CC0A89582E0C81619F40E943B5405C0D5
:101FC00093E0C91611F40E941F510E94C91A801B88
:101FD000910B805D974068F30E94F01983E0C8166A
:101FE00031F48EE00E94F94B87E00E94EC4B809127
:101FF000670987FF0BC085E00E94F94B89E00E94CA
:10200000EC4B8091670988730E94B5528091D80784
:102010008823F1F081E090E09093DA078093D9076C
:10202000A8E0B1E0EDE1F1E082E101900D92815094
:10203000E1F78091D807843119F40E942A2803C05F
:1020400086E10E940829882339F00E94C24F04C00B
:102050001092DA071092D90792E0C91649F48091DC
:10206000670986FF02C083E007C0C092690006C00E
:1020700023E0C21631F482E0809369001CBA81E04B
:102080008DBB10926F0910926E090E94C91A2C0123
:102090003E010894611C711C50EC352E46E0242E44
:1020A000A8950E940322823019F40E946F2009C073
:1020B000833019F40E94E32604C0843059F50E944D
:1020C0005024182F0E941C16112321F180916709BA
:1020D00090E087709070892BD1F4163091F4809144
:1020E00076098823A1F0A1E4B1E0EDE1F1E082E11D
:1020F00001900D928150E1F710924E0910927609ED
:1021000006C01B3121F480E490E00E94C40E812FB0
:102110000E94C24F82E0C81619F40E943B5405C0C9
:1021200093E0C91611F40E941F51F894A090860BF9
:10213000B090870B1092870B1092860B8090880BC3
:102140009090890B1092890B1092880B789421E063
:10215000A216B10429F081E08816910409F0F9C1B2
:10216000F8948091820B9091830BA091840BB09195
:10217000850B89839A83AB83BC837894C3010E94C7
:10218000091E009721F43092060181E0AEC0AFE253
:10219000B1E0FC0182E101900D928150E1F7809164
:1021A0000601803461F58091920B8823F9F48091C7
:1021B000330190913401892BC9F4809131019091C0
:1021C0003201892B99F480912F0190913001892B54
:1021D00069F489819A81AB81BC810197A109B10918
:1021E00089839A83AB83BC8382E043C08091920B46
:1021F000823009F053C081E08093920B4FC0803849
:1022000009F04CC08091920B882309F047C080915F
:10221000330190913401479709F040C0809131011A
:1022200090913201CB97D1F580912F01909130019F
:10223000CB97A1F589819A81AB81BC810196A11DC3
:10224000B11D89839A83AB83BC838091820B90916B
:10225000830BA091840BB091850B0196A11DB11D3C
:102260008093820B9093830BA093840BB093850B88
:1022700081E08093920BC3010E94091EAFE2B1E09E
:10228000FC0122E101900D922150E1F7892B31F4FC
:10229000309206011092890B1092880B89819A81E5
:1022A000AB81BC8120917701309178014091790117
:1022B00050917A01820F931FA41FB51F89839A83BF
:1022C000AB83BC83C3010E94091EADE1B1E0FC01F8
:1022D00082E101900D928150E1F78091920B813063
:1022E00039F4109206011092920B80937D010AC07E
:1022F0008091920B823031F48CE390E090931E0138
:1023000080931D0191E0A916B10409F0CEC00E948E
:10231000621E0E9435300E940B2A80919A0790918C
:102320009B07892B61F1809177099091780901973A
:10233000E1F40E948C0E7B018C011616170618061C
:1023400019064CF10E941833882311F00E94C24FE5
:10235000A3E5B1E0EDE1F1E082E101900D92815061
:10236000E1F782E00E94595016C0A3E5B1E0EDE12B
:10237000F1E082E101900D928150E1F709C0A3E5FF
:10238000B1E0EDE1F1E082E101900D928150E1F7E1
:10239000EE24FF248701D090670927E0D2228091A4
:1023A0007609882361F5DD20B1F40E94A70EAB0108
:1023B000BC0114161506160617062CF18091AD0403
:1023C0009091AE04A091AF04B091B0040097A10524
:1023D000B105C9F010C083E0D81689F48091940B40
:1023E000882369F40E94A70EAB01BC0114161506E0
:1023F0001606170644F081E08093760904C040E099
:1024000050E060E070E0809174098F5F8093740900
:102410008C33A9F41092740980917009909171091C
:10242000A0917209B09173090196A11DB11D80930D
:10243000700990937109A0937209B0937309809108
:102440006509882319F40E94E64D2FC0843019F4E1
:102450000E94C24C2AC0853021F592E0D91641F085
:1024600021E0D21629F080917609882309F4DFC192
:1024700080E00E94E54B80919A0790919B07892B01
:1024800061F08091770990917809019731F481E0AA
:10249000B801A7010E94784C08C081E00E94E54B7A
:1024A00004C0863011F40E94064C81E08816910425
:1024B00009F04FC080916709877029F410927D015F
:1024C00010927C010BC0833049F0813069F50E9485
:1024D000595010927D0110927C0126C080919C077A
:1024E00090919D0720917F09213019F4959587954A
:1024F0000BC0223049F4880F991F24E081309207E5
:102500001CF080E094E005C08034910514F480E470
:1025100090E00E94C40EA1E4B1E0EDE1F1E082E1BF
:1025200001900D928150E1F71092760980911B0184
:1025300090911C01019769F410921C0110921B01EB
:10254000A3E5B1E0EDE1F1E082E101900D9281506F
:10255000E1F780914E098823D9F00E948630182F28
:102560008823E1F080518B3058F4A1E4B1E0EDE133
:10257000F1E082E101900D928150E1F70E94D731A4
:1025800010924E0910927609812F0E94C24F06C008
:1025900010924D091092500910924F0980916709CD
:1025A0008770823080F40E947132182F882359F08E
:1025B00010924E091092760980E490E00E94C40EB9
:1025C000812F0E94C24F81E0A816B104F1F48091DE
:1025D000C204882359F08091D30481508093D3049E
:1025E000882321F480E090E00E9412248091D4049A
:1025F000882359F08091E50481508093E504882375
:1026000021F481E090E00E94122480916C09909165
:102610006D09019711F40E94C14E10926D0910923C
:102620006C090E94C91A84199509409708F49DC045
:102630000E94C91A2C010E944C1B0E945B1B88231C
:1026400009F493C0179A90916509843141F48091FF
:102650006609882309F089C00E94E55954C0813178
:1026600049F49F5F80911A01891708F0E4C09091A6
:102670006609E1C0823149F480916609981719F41E
:1026800090911A01D8C09150D6C08331A1F48091A5
:102690006609882339F497E09093660926E1209330
:1026A0001A01C9C0873079F587E18093660996E2FF
:1026B00090931A0122C0863189F480917709909114
:1026C0007809019709F051C00E941833882311F04E
:1026D0000E94C24F82E00E94595047C0883179F46D
:1026E00080916609873021F40E94AC4F97E0A3C027
:1026F000873109F0A0C00E94B74F97E19CC08F308E
:1027000041F40E946F1A1092660920921A0190E01B
:1027100092C0803151F5809167098770823088F4CA
:1027200080917609882309F58091AD049091AE04DB
:10273000A091AF04B091B0040097A105B105A9F034
:1027400002C0833091F481E0809376090EC0892F16
:1027500087500E94024D09C0873129F4892F875183
:102760000E94734D02C00E94C14E80917C0188235B
:1027700021F080917C01813099F481E090E0909388
:102780007809809377098091670987708250823039
:1027900028F41092060181E08093070115981DC06E
:1027A00080917C01833029F424E020937C0185E230
:1027B00008C080917C01823031F484E080937C01F8
:1027C00086E20E94C24F10927809109277093092E7
:1027D000060190E190930701159A80919A079091D4
:1027E0009B07892B41F08091770990917809019797
:1027F00011F4149801C0149A8091D807882371F0BD
:102800008091AD049091AE04A091AF04B091B0045A
:102810000097A105B10511F0139801C0139A0E9409
:10282000CC15813011F416983BCC169A39CC80E047
:102830000E94784C20CE909365098091660987307C
:1028400009F08ACF84CF8EBD0DB407FEFDCF089569
:102850002C988EBD0DB407FEFDCF1EBC0DB407FE37
:10286000FDCF8EB52C9A08952C988EBD0DB407FE21
:10287000FDCF1EBC0DB407FEFDCF8EB51EBC0DB442
:1028800007FEFDCF8EB52C9A08952C98805C8EBDE6
:102890000DB407FEFDCF6EBD0DB407FEFDCF2C9A23
:1028A00008950F931F93182F0E942814082F812F2B
:1028B0008F5F0E942814982F802F1F910F910895E9
:1028C0000F931F93182F0E943414082F812F8F5FAE
:1028D0000E943414982F802F1F910F9108950F9309
:1028E0001F93182F072F0E944514812F8F5F602F91
:1028F0000E9445141F910F9108952C9880588EBD09
:102900000DB407FEFDCF6EBD0DB407FEFDCF2C9AB2
:1029100008952C9880568EBD0DB407FEFDCF6EBD78
:102920000DB407FEFDCF2C9A08951F93182F8FE149
:1029300063E00E9489148FE1612F0E947D141F9132
:1029400008951F93182F82E00E94951484E1612F4F
:102950000E94451482E161E00E94451483E00E94D8
:1029600095148AE00E94341480FDFBCF82E00E941F
:10297000951482E160E00E94451488E10E94601491
:102980001F910895FF920F931F93F82E8B0182E001
:102990000E94951484E16F2D0E94451486E1B801D0
:1029A0000E946F1483E00E9495148AE00E94341400
:1029B00080FDFBCF1F910F91FF9008952C988AE323
:1029C0008EBD0DB407FEFDCF1EBC0DB407FEFDCFBE
:1029D0008EB52C9A08952C988AE38EBD0DB407FE0F
:1029E000FDCF1EBC0DB407FEFDCF9EB51EBC0DB4C1
:1029F00007FEFDCF8EB52C9A08952C988AE38EBDE4
:102A00000DB407FEFDCF1EBC0DB407FEFDCF9EB575
:102A10001EBC0DB407FEFDCF8EB51EBC0DB407FE67
:102A2000FDCF7EB51EBC0DB407FEFDCF6EB52C9A52
:102A30000895FC012C988AE38EBD0DB407FEFDCFEE
:102A400020E030E008C01EBC0DB407FEFDCF8EB5FF
:102A500081932F5F3F4F26173707A8F32C9A0895CD
:102A6000982F2C988AE78EBD0DB407FEFDCF9EBD32
:102A70000DB407FEFDCF2C9A0895282F2C988AE7D5
:102A80008EBD0DB407FEFDCF9EBD0DB407FEFDCF7C
:102A90002EBD0DB407FEFDCF2C9A0895282F2C983B
:102AA0008AE78EBD0DB407FEFDCF9EBD0DB407FEB7
:102AB000FDCF2EBD0DB407FEFDCF7EBD0DB407FECC
:102AC000FDCF6EBD0DB407FEFDCF2C9A0895FC011D
:102AD0002C988AE78EBD0DB407FEFDCF20E030E0D4
:102AE00008C080818EBD0DB407FEFDCF2F5F3F4F24
:102AF000319626173707A8F32C9ACB010895282F73
:102B00002C988AE78EBD0DB407FEFDCF80E090E0E3
:102B100005C02EBD0DB407FEFDCF019686179707A1
:102B2000C0F32C9A08958FE160E00E94451480E183
:102B300060E070E00E946F1482E16FEF7FE10E941D
:102B40006F148AE06FEF7FE10E946F1483E00E94B0
:102B5000951487E067E00E94451487E00E942814DE
:102B600080FDFBCF87E062E00E9489148FE160E383
:102B70000E947D148FE10E94281485FDFBCF80E028
:102B80000E94951486E10E94511420E08750984FCE
:102B900009F421E0822F089581E00E94A114969506
:102BA000879596958795817008958FE10E942814E6
:102BB0008095881F8827881F0895EF92FF920F93B2
:102BC0001F938C0180E00E94951480E00E946014A5
:102BD000F82EE92E60911704709118046A5F7F4FF8
:102BE000600F711F89E1683D780710F0685D7941D9
:102BF00080E00E946F148F2D9E2D1F910F91FF90EA
:102C0000EF900895EF92FF920F931F938C0180E055
:102C10000E94951482E00E946014F82EE92E07525B
:102C2000164E82E0B8010E946F148F2D9E2D1F91C9
:102C30000F91FF90EF9008950F931F930091190447
:102C400010911A040150104080E00E9495148EE10A
:102C500060E40E947D14B80189E1083D180710F076
:102C600067ED79E18CE00E946F141F910F91089538
:102C70001F93CF93DF9381E00E94951489E10E9416
:102C80002814182F80E00E9495148EE00E942814CA
:102C9000C82FD0E081E00E94951489E10E94281499
:102CA000181779F78CE00E9451149F718C179D07BB
:102CB00020F49C012952364E09C0C817D90719F4CF
:102CC00027ED39E105C09C01215030402C1B3D0B04
:102CD000C901DF91CF911F910895A7E0B0E0E3E72C
:102CE000F6E10C9491628C01E0901C04F0901D04BC
:102CF000E80EF91E82E0B8010E946F1480E00E9485
:102D0000301584E0B8010E946F1486E0B7010E947C
:102D10006F148FE160E80E947D148FE160E80E94EB
:102D200089148CE16AE00E9489148FE168E00E94B6
:102D30007D1480911B048550823008F068C000E04B
:102D400010E08CE10E9428148A7031F40F5F1F4F4D
:102D500083E0083E1807A9F78CE10E94281481FD42
:102D600005C083E0083E180708F451C08FE168E011
:102D70000E94891480E00E9460145C0186E00E9439
:102D800060146C010894C11CD11C80E0B6010E9443
:102D90006F148E010F5F1F4FC80167E070E00E9443
:102DA0001915EE24F02E012F8CE10E94281481FFCA
:102DB0002AC08C8185FF27C08FE160E80E947D14C6
:102DC0008FE160E80E9489148CE16AE00E94891416
:102DD0008FE168E00E947D148CE10E9428148A70C3
:102DE000D9F38FE168E00E94891480E0B6010E9467
:102DF0006F148F2D902F67E070E00E941915E394F7
:102E000080E1E81689F680E0B5010E946F142796EC
:102E1000EAE00C94AD62A0E0B0E0E1E1F7E10C94EF
:102E20009262B82E282F392F6901EE24FF248701E2
:102E300011C00E94DE14D82F0E94DE14C82FCE01CC
:102E4000A0E0B0E0E80EF91E0A1F1B1F8EEF9FEFF7
:102E5000C80ED91E92E0C916D10458F7C701D8018F
:102E60009C01AD01B0FE0BC00E94DE14D82FC0E063
:102E70009E0140E050E02E0D3F1D401F511F2030AD
:102E800080E0380781E0480780E05807A0F0CA01D9
:102E900040E050E0A0E0B0E0280F391F4A1F5B1F60
:102EA000203090E0390791E0490790E0590718F089
:102EB000C90101969C01C901CDB7DEB7E9E00C94C8
:102EC000AE620F931F938B010E94DD15C8010E9413
:102ED0000B179C0120953095C9011F910F91089502
:102EE000EF92FF920F931F938C017B0180E00E9471
:102EF00095140752164E80E0B8010E946F14C70166
:102F00000E940B179C0120953095C9011F910F91CC
:102F1000FF90EF900895A0E0B0E0E1E9F7E10C94B4
:102F200093626C017B018A014115510509F444C08B
:102F30004130510551F40E94DD15C7010E9402166F
:102F40000E94DE140E94301537C080E00E94951464
:102F5000C0911704D09118042696CC0DDD1D89E18F
:102F6000C83DD80710F0C85DD94180E1BE010E947C
:102F70006F14B801615070406C0F7D1F99E1683D7E
:102F8000790710F0685D794182E10E946F1489ED44
:102F900099E1E80EF91E84E1B7010E946F148FE1F8
:102FA00060E10E9489148FE160E20E947D148FE14C
:102FB0000E94281485FDFBCFCDB7DEB7E8E00C9466
:102FC000AF628FE164E00E9489148DE10E942814B1
:102FD00082FDFBCF8FE10E94281487FDFBCF8EE19D
:102FE00060E20E947D1408951F93182F83E00E94D1
:102FF000951485E1612F0E9445141F91089583E087
:103000000E94951485E10E9428140895FC012C98D3
:103010008AE38EBD0DB407FEFDCF20E030E00AC08C
:103020001EBC0DB407FEFDCF8EB581932F5F3F4FC1
:10303000841719F02617370798F310822C9AC901C4
:1030400008950F931F93CF93DF938C01C0E0D0E0DE
:1030500003C00E94DE142196C017D107D0F3DF9180
:10306000CF911F910F910895CF93DF93EC010E94B0
:10307000F762AC012C988AE78EBD0DB407FEFDCF38
:1030800020E030E00AC0FE01E20FF31FE491EEBD44
:103090000DB407FEFDCF2F5F3F4F2417350798F380
:1030A0002C9ACA01DF91CF9108958EE160E20E94CF
:1030B000891480E190E00E94C21A8DE10E942814D8
:1030C00083FDFBCF80FFF9CF8FE164E00E947D1488
:1030D00008951F938EE160E20E94891480E190E0E0
:1030E0000E94C21A5E9880E190E00E94C21A5E9A25
:1030F00080E190E00E94C21A1FEF2C981EBD0DB413
:1031000007FEFDCF2C9A80E190E00E94C21A8DE16B
:103110000E94281483FDF1CF80FFEFCF8FE160EC98
:103120000E9445148EE160E80E94451488E060E04A
:1031300070E00E946F148CE067ED79E10E946F14DB
:103140008AE067ED79E10E946F1484E068ED79E12F
:103150000E946F1481E00E94951488E161EA0E9448
:10316000451482E00E94951480E06DE00E944514B1
:1031700081E060E00E94451482E062E30E94451411
:103180008AE06EEE75E00E946F1486E062E17CE0FA
:103190000E946F1484E062E10E94451483E060E4C1
:1031A0000E94451489E06FE30E94451483E00E9469
:1031B000951485E160E00E94451484E0609100016F
:1031C0000E94451485E0609101010E94451482E04F
:1031D000609102010E94451483E0609103010E9406
:1031E000451480E0609104010E94451481E06091E3
:1031F00005010E94451482E10E9428148F7180937A
:103200001B0480E060E070E00E94C21480E160E096
:1032100071E00E94C21484E162E774E00E94C2146B
:1032200080E00E9495148FE164E00E9445141F9194
:103230000895CF93DF93EC0181E00E94951489E11A
:103240000E942814882321F40E94951480E044C031
:1032500080E00E9495146091190470911A0480E036
:103260000E946F148091190490911A04909318048D
:103270008093170481E194E066E070E00E941915E4
:10328000809112048F7180931204809114048F71C5
:1032900080931404209111043091120430931A0485
:1032A0002093190480911304909114048F5E95402B
:1032B00080F489E1283D380760F420FD0AC0809140
:1032C000160487FD06C08091150484FD02C087FDA9
:1032D00006C00E94691882E0DF91CF910895F894AA
:1032E0008091820B9091830BA091840BB091850B00
:1032F00080938A0790938B07A0938C07B0938D07D8
:103300008091800B9091810B90939307809392070B
:103310007894CE016EE070E00E94191581E0DCCF58
:1033200098B18F70907F892B88B90895469898B18D
:103330008F70907F892B88B90000449A83E090E0D9
:103340000E94C21A449808951F93182F88B1912F94
:1033500092959F70807F982B98B9449A83E090E073
:103360000E94C21A449888B11F70807F812B88B94F
:10337000449A83E090E00E94C21A44981F910895F5
:10338000469A0E94A419089546980E94A419089587
:103390000E94C01981E090E00E94C21A0895CF9364
:1033A000DF93EC0103C021960E94C819888188230D
:1033B000D1F7DF91CF91089580E10E94C41981E097
:1033C00090E00E94C21A0895882311F48CE001C095
:1033D0008EE00E94C41981E090E00E94C21A089514
:1033E00081E00E94C41989E190E00E94C21A089508
:1033F000662349F0613011F4805C05C0623011F43D
:103400008C5E01C08C5A80680E94C41981E090E0F3
:103410000E94C21A08950F931F93042F0E94F81957
:1034200010E004C080E20E94C8191F5F1017D4F397
:103430001F910F910895682F80E040E10E940B1AC0
:103440000895CF93DF93EA010E94F81903C00E9408
:10345000C8192196FE0184918823C9F7DF91CF9185
:1034600008950F931F938A010E94F819C8010E94C2
:10347000CF191F910F9108951F93142F0E94F819CF
:10348000812F0E94C01981E090E00E94C21A1F9112
:1034900008950F931F93CF93DF938B01880F880FAD
:1034A000880F887380640E94C419C0E0D0E081E076
:1034B00090E00E94C21A81E090E00E94C21AF801D6
:1034C000EC0FFD1FE4918E2F0E94C0192196C83089
:1034D000D10569F7DF91CF911F910F9108951F9347
:1034E000CF93DF9388E290E00E94D11A83E00E949C
:1034F000961982E490E00E94C21A83E00E94961915
:1035000081E090E00E94C21A83E00E94961981E057
:1035100090E00E94C21A82E00E94961981E090E039
:103520000E94C21A88E20E94C41981E090E00E94C1
:10353000C21A88E00E94C41981E090E00E94C21A79
:1035400081E00E94C41989E190E00E94C21A86E0DD
:103550000E94C41981E090E00E94C21A8CE00E948F
:10356000C419C4ECD0E010E0FE0165917491812F84
:103570000E94491A1F5F22961830B1F7DF91CF9150
:103580001F91089528EC00002A95E9F70197D1F7DB
:103590000895F8942091BC023091BD027894C9013D
:1035A0000895AC01F8942091BC023091BD0278944A
:1035B00001C0A895F8948091BC029091BD027894C6
:1035C000821B930B84179507A0F30895DC01F894F0
:1035D0007894809189038823A9F0F894E091870377
:1035E000F0E0E95FFC4F80818C93809187038F5FCF
:1035F0008F7780938703809189038150809389031B
:10360000789481E00895A1E0B0E0E9E0FBE10C945A
:1036100097628E010F5F1F4F01C0A895C8010E94DD
:10362000E61A8130D1F32196E4E00C94B362A1E074
:10363000B0E0EDE1FBE10C949962CE0101960E94AD
:10364000E61A882311F490E022C020910A042F3753
:1036500010F490E005C010920E0410920D0492E058
:103660008981E22FF0E0E657FC4F8083E22FEF5F85
:10367000E0930A048A3059F4F0E0E657FC4F1082D8
:1036800010920A0410920E0410920D0491E0892FFA
:103690002196E2E00C94B5629091C20283B1EEEB08
:1036A000F2E0E90FF11D80958F7080839F5F93702A
:1036B0009093C20208959091BF028091BE02982318
:1036C0008091C00298238091C102982341F19830E3
:1036D00011F494E11DC0943011F493E119C09230BB
:1036E00011F492E115C0913011F491E111C09C30B8
:1036F00011F498E10DC0933011F49FE009C09930A6
:1037000011F490E105C09A3011F090E001C096E10B
:103710008091950B981729F09093950B03C0109208
:10372000950B90E0892F0895EF92FF920F931F93CE
:10373000CF93DF93F894E090BC02F090BD027894B0
:103740008701A895F894C091BC02D091BD027894ED
:10375000CE01801B910B409718F00E944C1B8E01EC
:103760000E945B1B882331F4CE19DF09C051D74278
:1037700040F389E1CDB7DEB7E6E00C94B1620F9378
:103780001F93CF93DF939C01EB018A0101C0A895A1
:10379000F999FDCFCE01B9014FE150E00E948D6350
:1037A0001F8E8881992787FD90950E94C062892B82
:1037B00021F4CE01B8010E94F062DF91CF911F91F8
:1037C0000F9108950F931F93CF93DF939C01EB010B
:1037D0008A0101C0A895F999FDCFCE01B9014FE04A
:1037E00050E00E948D631F868881992787FD909500
:1037F0000E94C062892B21F4CE01B8010E94F062C0
:10380000DF91CF911F910F910895EF92FF920F9347
:103810001F93142F052FF62EE72E01C0A895F999B6
:10382000FDCF0E949D639B01AC012F3F8FEF3807B6
:103830008FEF48078FEF580741F4212F302F4F2D7E
:103840005E2DC901DA019C01AD01B901CA011F91C8
:103850000F91FF90EF9008951F93CF93DF93EC01AA
:103860000E94F762182F813414F58091050390911E
:103870000603019711F4A895FECF81E090E09093A4
:1038800006038093050383EC92E0BE010E94F06280
:103890008091C3028093C60011501093040381E00D
:1038A000809303038091C10080668093C100DF9103
:1038B000CF911F9108951F93BC01FC01019000203E
:1038C000E9F731971E2F181B11340CF58091050371
:1038D00090910603019711F4A895FECF81E090E046
:1038E000909306038093050383EC92E00E94696342
:1038F0008091C3028093C60011501093040381E0AD
:10390000809303038091C10080668093C1001F9162
:1039100008951F93482F792F162F613444F5809115
:10392000050390910603019711F4A895FECF81E05D
:1039300090E0909306038093050323EC32E0E62F9A
:10394000FF27E7FDF095C901642FAF010E942863AE
:103950008091C3028093C60011501093040381E04C
:10396000809303038091C10080668093C1001F9102
:1039700008950000000008952D9A2F98000000007F
:103980002F9A90E087FF02C02D9A01C02D982F98A2
:10399000000000002F9A9F5F983011F0880FF2CF3F
:1039A00008951F93CF93DF93182FEB01809110049C
:1039B000813021F4CB010E94513EEC01F8942F9A02
:1039C0005F9A80E30E94BC1C5F982F9A5F9A1F73D6
:1039D000812F80640E94BC1C80E0D7FF02C02D9A1A
:1039E00001C02D982F98000000002F9A00000000C1
:1039F0008F5F803119F0CC0FDD1FEFCF5F982D98CE
:103A00005F9A000000001E9BFECF5F985F9878943D
:103A1000DF91CF911F9108951F93CF93DF93C0E063
:103A2000D1E012E0688179812296812F0E94D11C19
:103A30001F5F1530B9F7DF91CF911F910895FF9265
:103A40000F931F93182F062FF72EBA010E94D11C37
:103A5000812F8F5F602F7F2D0E94D11C1F910F91AE
:103A6000FF900895F8942F9A5F9A8F7380680E9450
:103A7000BC1C80E020E030E02F98000000002F9A6E
:103A800000000000220F331F1E9921608F5F8031DC
:103A900099F7932F5F98789480911004813021F4E6
:103AA000822F0E94513E9C01C90108951F93CF931C
:103AB000DF9380E00E94321D8050904419F481E031
:103AC0008093100482E00E94321D8F5F9F4F61F04F
:103AD00012E0C0E0D1E0812F0E94321D88839983DB
:103AE00022961F5F1530B9F7DF91CF911F9108958E
:103AF0009F92AF92BF92CF92DF92EF92FF920F937D
:103B00001F93182F042FB52EA62E972E0E94321D1C
:103B10006C01812F8F5F0E94321D7C018FEFC816D0
:103B20008FEFD8068FEFE8068FEFF80641F4202FCD
:103B30003B2D4A2D592DC901DA016C017D01B601D9
:103B4000C7011F910F91FF90EF90DF90CF90BF9032
:103B5000AF909F9008951F1D1F1E1F1E1F1F1E1F29
:103B60001E1FCF93DF93EC012C964AE834D06627D2
:103B7000772736E4AEE6B1E0532F537009F0119782
:103B8000321729F078F56A0F7B1F3395F3CF4CE09D
:103B900022D0E6E5FBE330E0C8953196313011F4F0
:103BA00051110A94321720F4600D711D3395F4CF32
:103BB000402D439510D02150A8F0620F711D882729
:103BC000992748E108D015D04CE305D012D02CE35A
:103BD00002D00FD00BC03A912A912417310540F042
:103BE0000F900F906FEF7FEF8FEF9FEFDF91CF91EF
:103BF000089551E2AA1B08F4A40FA79597958795FD
:103C0000779567955A95B9F7620F711D811D911DC2
:103C10000895CF93DF93FC0120813181428153814C
:103C2000CC27DD2757FD3CC0C6E9DBE06CE33CD088
:103C30000882198239D00A821B8268E135D00C8251
:103C40001D82F9012C5F3F4F67E02ED00C861D8648
:103C50009F01A6E4EEE6F1E0BA2FB37009F03197C8
:103C60002E173F0720F02E1B3F0BA395F3CFAA87FB
:103C70001B862E873F87E6E5FBE3AA27C89531968A
:103C8000A13011F4B1110A942015310520F020194A
:103C90003109A395F3CFA887198623952E833F83F7
:103CA000CE01DF91CF910895002470E2220F331FDF
:103CB000441F551F001C061610F0061A23957A950E
:103CC000A9F70895EEE4F4E08281813041F4808127
:103CD0009181019791838083892B09F412823D960B
:103CE00084E0E63BF80781F70895CF92DF92EF92E8
:103CF000FF920F931F936B017C018AE290E09093F7
:103D00001D0480931C0480E00E94951482E06DECF9
:103D10007FE10E946F148FEF66E070E00E947F15D4
:103D200000E011E0C80166E070E00E94671586E0DF
:103D300098E00E943D1581E090E00E943D1580E0F2
:103D400098E00E943D1586E00E94301584E00E94B4
:103D5000301581E090E00E943D15C80166E070E0FA
:103D60000E9467156091AD047091AE048091AF041C
:103D70009091B0040E944E1580E066E070E00E94D1
:103D80007F15C701B6010E944E158CEC9FE10E9481
:103D90006D161F910F91FF90EF90DF90CF900895D7
:103DA000EF92FF920F931F93CF93DF937B018C01D0
:103DB000E901E4E4F4E020E080819181A281B38113
:103DC0008E159F05A007B10711F4922F0DC02F5F2C
:103DD0003D96283089F7CD2BF9F09091AC04892FCE
:103DE0008F5F87708093AC048DE0989FF001112461
:103DF000EC5BFB4FEF012496DA0186E00D9009920F
:103E00008150E1F7E082F1820283138380EB94E03A
:103E10009387828781E08487CDB7DEB7E6E00C9494
:103E2000B162ACE1B0E0E7E1FFE10C948F62CE015A
:103E300001966CE170E00E9419158F8198850E94AF
:103E4000513E4C016F85788989899A890E94553E37
:103E50005B016C01698D7A8D8B8D9C8D0E94553E26
:103E60007B018C0189819A810E94513E019709F062
:103E700071C08B819C810E94513E8050984009F016
:103E800069C08091AD049091AE04A091AF04B0914F
:103E9000B004E816F9060A071B0709F05BC0CE015B
:103EA000439660E071E046E050E00E947063009746
:103EB00009F050C0AE14BF04C006D10611F482E070
:103EC0004AC08E01075F1F4FC601B501A80121E05E
:103ED00030E00E94D01E81E088169104D9F58CE173
:103EE00090E090931D0480931C048EE090E00E946B
:103EF000021681E090E00E943D1580E098E00E946B
:103F00003D1586E00E94301584E00E94301582E065
:103F100090E00E943D1580E091E066E070E00E9434
:103F200067156091AD047091AE048091AF049091DB
:103F3000B0040E944E15C80166E070E00E9467154B
:103F4000CE010F9664E070E00E94671586E098E06D
:103F50000E94192080E06C96ECE00C94AB62EF922A
:103F6000FF920F931F93E0902404F090250400919A
:103F70002604109127042091B1043091B20440919D
:103F8000B3045091B404DA01C9018E299F29A02BF2
:103F9000B12B8F5F9F4FAF4FBF4F49F48EE194E03D
:103FA0006FEF70E046E050E00E94436335C08091BF
:103FB000AD049091AE04A091AF04B091B0048E25F1
:103FC0009F25A027B12782239323A423B5230097FD
:103FD000A105B10511F421E009C0E090B504F0900D
:103FE000B6040091B7041091B80422E0E4E4F4E0D0
:103FF0008485813099F480819181A281B3818E156D
:104000009F05A007B10751F4AEE1B4E0349686E015
:1040100001900D928150E1F720E005C03D9684E0CB
:10402000EC3AF80729F7822F1F910F91FF90EF903C
:1040300008950F931F938C0180911C0490911D048F
:104040000E9690931D0480931C0480E090E00E94E3
:1040500002168EE194E066E070E00E94671580E051
:1040600091E066E070E00E946715C8010E943D156E
:1040700088ED99E10E946D161F910F910895AEE0B1
:10408000B0E0E5E4F0E20C949862CE0101960E9463
:1040900019198823F1F0AEE1B4E0FE01379686E00D
:1040A00001900D928150E1F78D859E850E94513ED1
:1040B00028E08030920711F411E00CC0865098403F
:1040C00031F40E94111F182F0E941C1603C00E9479
:1040D0001C1610E0812F2E96E3E00C94B462A8E049
:1040E000B0E0E5E7F0E20C94976282E290E00E9493
:1040F000DD15CE01019668E070E00E9419158981F6
:104100008093BC048A818093BD0460911C047091EB
:104110001D0482E290E00E946117892B81F08AE3FE
:1041200090E00E94DD150E94FD146093BE04709320
:10413000BF048093C0049093C10487E057C080916E
:10414000BC04883031F16D817E818F8198850E9419
:10415000553E9B01AC016093BE047093BF048093F5
:10416000C0049093C1048091BC04833019F40E9470
:1041700069183BC08530C9F58091BD048130A9F52F
:104180002093B5043093B6044093B7045093B80419
:104190002CC040911C0450911D0482E290E062E228
:1041A00070E00E948B1782E290E00E94021680E08D
:1041B0000E94301580E00E94301580E090E00E945F
:1041C0003D1560911C0470911D0482E290E00E94F4
:1041D00070178C0184E290E00E940216C8010E94D0
:1041E0003D1581E00E94542101C08AE02896E4E058
:1041F0000C94B362A0E0B0E0E0E0F1E20C949262D3
:10420000B82EEB016A01E8E3F4E0EE24FF24870115
:10421000308121813296C901A0E0B0E0E80EF91E9C
:104220000A1F1B1F84E0E434F80791F781E0B816F9
:1042300051F480E00E949514C752D64E80E0BE0132
:104240000E946F1403C0CE010E94DD15C6010E94BA
:104250000B179C0140E050E02E0D3F1D401F511FE9
:10426000203080E0380781E0480780E05807A0F060
:10427000CA0140E050E0A0E0B0E0280F391F4A1F1B
:104280005B1F203080E0380781E0480780E0580756
:1042900018F0C90101969C0120953095C901CDB750
:1042A000DEB7E9E00C94AE62ACE1B0E0EAE5F1E241
:1042B0000C949762182F80911C0490911D044496D1
:1042C00090931D0480931C048EE090E00E940216DF
:1042D00080E095E40E943D1580911C0490911D049E
:1042E0000E943D158091B9049091BA040E943D1539
:1042F00080E090E40E943D1580E40E943015812FFB
:104300000E94301580E090E00E943D156091AD0460
:104310007091AE048091AF049091B0040E944E154C
:1043200060912404709125048091260490912704C3
:104330000E944E158EE090E064E170E00E947017DC
:104340008C0188E190E00E940216C8010E943D1590
:104350000E94AF1F882309F443C0DE011196ECE1EF
:10436000F4E09CE101900D929150E1F7823049F424
:104370006091B5047091B6048091B7049091B8042F
:1043800008C06091240470912504809126049091C6
:1043900027040E94751E0E941C160E94C91A8C01D7
:1043A000A8950E943F20882311F00E941C160E94AD
:1043B000AF1F882311F420E008C00E94C91A801B97
:1043C000910B8858934160F326E0ACE1B4E0FE0124
:1043D00031968CE101900D928150E1F7222329F46E
:1043E00080E098E00E94192020E08091B90490912B
:1043F000BA0401969093BA048093B904822F6C9604
:10440000E4E00C94B362A4E1B0E0E9E0F2E20C94E1
:1044100095620E943F20882309F4A1C0823011F4E4
:1044200085E09DC08EE090E064E170E00E9461173D
:10443000892B09F091C08EE090E00E94DD15CE013D
:10444000019664E170E00E94191569897A898B8967
:104450009C890E94553E7B018C012091B1043091D2
:10446000B2044091B3045091B4048981682F70E084
:10447000CB01807F90708034910509F06DC08091F0
:10448000AD049091AE04A091AF04B091B004E816D1
:10449000F9060A071B0799F02E293F29402B512BBB
:1044A0002F5F3F4F4F4F5F4F51F08FEFE8168FEF69
:1044B000F8068FEF08078FEF180709F04DC06F70EF
:1044C0007070660F771F660F771F6093BB048B8138
:1044D0009C810E94513E2091BB04821B91099093C4
:1044E0001D0480931C046D857E858F8598890E94AC
:1044F000553E609324047093250480932604909382
:104500002704E0922804F092290400932A041093CF
:104510002B048091BB04853120F0845190E00E94EF
:1045200021186091240470912504809126049091B3
:1045300027044EE154E020E030E00E94D01E8A853E
:10454000813011F482E00BC0813111F483E007C0A7
:10455000863011F484E003C00E941C1680E064964B
:10456000E6E00C94B162A0E0B0E0E9EBF2E20C947A
:104570009462D82EEB017A0184E190E0E80EF91EF6
:10458000F0921D04E0921C048CEE9FEFE80EF91EE1
:1045900082E290E00E9402168D819E810E943D156C
:1045A0008F8198850E943D1569857A858B859C85CC
:1045B0000E944E156D857E858F8598890E944E15C7
:1045C00080E50E9430158D2D8F730E94301584EB8D
:1045D00095E00E943D1560E070E080E090E00E9470
:1045E0004E156091AD047091AE048091AF0490912E
:1045F000B0040E94553E6093380470933904809350
:104600003A0490933B0469817A818B819C810E945A
:10461000553E60933C0470933D0480933E04909318
:104620003F041092400486E08093410480911C0472
:1046300090911D040E94513E909343048093420444
:1046400040911C0450911D0481E062E270E00E94E0
:10465000FA208C0182E390E00E940216C8010E94B9
:104660003D1586E00E945421682F882301F58D2D89
:1046700090E083709070892B41F089859A85AB8595
:10468000BC850196A11DB11D0EC0E114F10479F0A5
:10469000970140E050E089859A85AB85BC85820F03
:1046A000931FA41FB51F89879A87AB87BC87862F66
:1046B000CDB7DEB7E7E00C94B062A2E1B0E0E3E68C
:1046C000F3E20C94996220912C0430912D04C901DD
:1046D000A0E0B0E08A839B83AC83BD8380912E04ED
:1046E00090912F049F838E83398728871A861B8693
:1046F0001C861D868091340490913504A091360467
:10470000B09137040196A11DB11D8E879F87A88B9C
:10471000B98B84E0BE016F5F7F4F40E050E00E94A4
:10472000B3226296E2E00C94B562A8E0B0E0EBE957
:10473000F3E20C948F627C018091300490913104FB
:104740000E94DD1500E010E06E010894C11CD11C30
:104750002EEEA22E26E0B22EAE0CBF1C92E0892EC9
:104760009924939453C0C60165E070E04AE00E942A
:104770000618080F191FC60169ED70E00E94E76274
:10478000892B91F4E114F10419F08AEE95E002C04E
:104790008AEE94E06BEF70E04AE00E940618080F82
:1047A000191FF501908232C0C60164ED70E044E04B
:1047B00050E00E940063892B19F4F501808226C025
:1047C00089818D30E1F48A818A30C9F48091320484
:1047D0009091330408171907C8F0EE0CFF1C8AEEFD
:1047E00096E0E80EF91E81E090E0F7019183808366
:1047F00015C00F5F1F4F0E94DE148A3039F0809180
:104800003204909133040817190798F38091320409
:10481000909133040817190708F4A5CF2896ECE007
:104820000C94AB62CF93DF93EC01009719F02AEE62
:1048300035E002C02AEE34E0FE01EE0FFF1FDF017B
:1048400043E0AA0FBB1F4A95E1F7AE0FBF1FAE535F
:10485000BB4F1C9211961D921D921D921C92149793
:1048600016961C921E92159718961C921E921797D8
:104870001D961D921D921D921C92509780E091E012
:10488000D901AC011D9241505040E1F7E651F94F7A
:1048900011821082C251D94F1882DF91CF910895B1
:1048A000A6E2B0E0E6E5F4E20C948B620091BB0472
:1048B00010E0025F1F4FCE01439664E170E00E945A
:1048C00019158B899C890E94513E90932D048093E9
:1048D0002C048D899E890E94513E90932F048093D1
:1048E0002E046F89788D898D9A8D0E94553E609334
:1048F00034047093350480933604909337042F8DDD
:104900002695269530E0C801820F931F90933104BD
:104910008093300480911C0490911D04821B930BA2
:1049200090933304809332046091240470912504A1
:1049300080912604909127040E94553E609338048C
:104940007093390480933A0490933B046091280457
:104950007091290480912A0490912B040E94553E65
:1049600060933C0470933D0480933E0490933F0415
:104970001092400486E08093410480911C04909141
:104980001D040E94513E9093430480934204409141
:104990001C0450911D0480E0B8010E94FA20892B6C
:1049A00009F099C198A1992309F495C16090240454
:1049B000709025048090260490902704E0902C04A9
:1049C000F0902D04A0902E04B0902F0402EC14E07F
:1049D000CC24DD246FEF7FEF2E010894411C511C85
:1049E000D201F80182E101900D928150E1F7AE8190
:1049F000BF81E885F9852A813B814C815D81898170
:104A0000882331F48FEF6F3F780711F4B6010BC0A4
:104A1000261537054805590531F4EE15FF0519F43B
:104A2000AA15BB05C1F00894C11CD11C0E5E1F4F16
:104A3000E2E0CE16D104A1F6FFEF6F3F7F0741F011
:104A40006B01C094D0948CE9C8168FEFD80619F486
:104A50000E945D23FFC0D7FE47C091FF3FC18091F8
:104A6000E6049091E704A816B90609F037C1C0948E
:104A7000D094C601880F991F8C0143E0000F111FCD
:104A80004A95E1F7080F191F0E531B4FF801618279
:104A9000728283829482B682A582F086E78281E068
:104AA00080830E94E03DF801618772878387948745
:104AB0008091340490913504A0913604B09137046C
:104AC0000196A11DB11D85879687A787B08B8CE3C2
:104AD000818B82E1B80140E050E00E94B322F82EC1
:104AE000882309F4FCC053C091FF03C00E945D23DA
:104AF0004DC092FF0FC0B601660F771FCB0123E0B8
:104B0000880F991F2A95E1F7680F791F6E537B4F25
:104B100084E038C090FF3FC0C601880F991F8C0108
:104B2000B3E0000F111FBA95E1F7080F191F0E53DC
:104B30001B4FF80120818091340490913504A0919D
:104B40003604B09137040196A11DB11D8587968763
:104B5000A787B08B223079F480E1B80140E050E0C3
:104B60000E94B32281E1B80140E050E00E94B322EC
:104B7000F82E85E0A1C0233019F0263009F0AEC030
:104B800080E1B80140E050E00E94B322F82EC60157
:104B90000E941224A4C093FF5FC0809132049091C0
:104BA0003304009711F480E055C05601AA0CBB1CD9
:104BB0008501F3E0000F111FFA95E1F70A0D1B1DA7
:104BC0000E531B4FF8012081213019F482E08083BD
:104BD00002C0223011F0FF243CC0A0E0B0E02091E0
:104BE0003404309135044091360450913704820FDB
:104BF000931FA41FB51FF80185879687A787B08BE1
:104C0000258136818091E6049091E70428173907C1
:104C1000B1F480E1B80140E050E00E94B322F82EE8
:104C2000C6010E949523F501E651F94F80819181DB
:104C3000019779F4C6010E943C45F82E0AC081E133
:104C4000B80140E050E00E94B322F82E83E0F80162
:104C500080838F2DF82E43C094FF40C0C601880F7B
:104C6000991F8C0173E0000F111F7A95E1F7080F6F
:104C7000191F0E531B4FF8018081813011F482E01F
:104C800022C08230E1F48091320490913304892B68
:104C900059F080E1B80140E050E00E94B322F82EC4
:104CA000C6010E9495231BC081E1B80140E050E09D
:104CB0000E94B322F82E83E0F801808310C0833075
:104CC00021F486E0F801808309C0853039F4C601FB
:104CD0000E94122403C068E0F62E01C0FF248F2D2D
:104CE000A696E0E10C94A762CF93DF930896909389
:104CF0001D0480931C0482E290E00E9402168091C1
:104D00002E0490912F040E943D1580912C049091C7
:104D10002D040E943D1580911C0490911D040E9459
:104D20003D1580E090E00E943D156091AD047091CA
:104D3000AE048091AF049091B0040E94553E609300
:104D400038047093390480933A0490933B04609143
:104D500024047091250480912604909127040E94D8
:104D6000553E60933C0470933D0480933E049093C1
:104D70003F041092400481E18093410480911C041F
:104D800090911D040E94513E9093430480934204ED
:104D900040911C0450911D0481E062E270E00E9489
:104DA000FA20EC01009711F4CFEFDFEF88E290E0FA
:104DB0000E940216CE010E943D1581E10E945421FD
:104DC000DF91CF910895A0E1B0E0E9EEF6E20C9416
:104DD0009562CE01099668E070E00E9419158985F8
:104DE0009A850E94513E90932D0480932C048B85CC
:104DF0009C850E94513E90932F0480932E048D85B4
:104E00009E850E94513E8C0108501040109333043F
:104E100000933204085F1F4F8091BB04E82EFF24EB
:104E20008EE090E0E80EF91E8F859889892BB9F104
:104E300060912404709125048091260490912704A8
:104E40000E94553E609338047093390480933A046D
:104E500090933B04609128047091290480912A0466
:104E600090912B040E94553E60933C0470933D0446
:104E700080933E0490933F041092400481E180931C
:104E800041048D859E85909343048093420480E085
:104E9000B701A8010E94FA20892B09F04AC0C70176
:104EA0000896909331048093300420912E04309121
:104EB0002F042B37310519F40E94D0333DC0253221
:104EC000310519F40E94A03B37C044E0203034077C
:104ED00019F40E94422D30C02434310519F40E9487
:104EE000022B2AC02938310519F40E948A2E24C0C9
:104EF0002151374201F50E94DD158E010F5F1F4FD2
:104F0000C80167E070E00E941915C80168EE70E002
:104F100047E050E00E940063892B69F48AE290E048
:104F20000E9402168FED90E00E9434180E947426B1
:104F3000FFCF89E001C080E06096E6E00C94B162AA
:104F40008091AD079091AE07A091AF07B091B007E7
:104F50008093240490932504A0932604B0932704FF
:104F600083E490E090932D0480932C0484E490E0FB
:104F700090932F0480932E048AE290E00E94021600
:104F800060E076E081E091E00E944E150E94E03DF5
:104F90006093C1077093C2078093C3079093C407BF
:104FA0000E944E1580E090E00E943D1580E090E068
:104FB0000E943D1560E070E080E090E00E944E1598
:104FC00080E06CE070E00E947F1580E091E066E098
:104FD00070E00E94671580E06AEC70E00E947F1527
:104FE00063E673E582E893E60E944E1581E095E35F
:104FF0000E943D1584E00E94301582E30E94301526
:1050000084E00E9430156091AD047091AE048091EF
:10501000AF049091B0040E944E1586E30E943015B3
:1050200084E00E9430156091AD077091AE078091C9
:10503000AF079091B0070E944E158FEF0E94301578
:1050400080E06CE270E00E947F158CE291E00E94AB
:10505000742608950F931F9381E08093D8078FEFF4
:105060009FEFAFEFBFEF8093240490932504A093AC
:105070002604B093270483E490E090932D0480935A
:105080002C0484E490E090932F0480932E041092DB
:10509000B1041092B2041092B3041092B4041092AE
:1050A000AD041092AE041092AF041092B0041092AE
:1050B00061091092620910926309109264091092BA
:1050C000B5041092B6041092B7041092B80410926E
:1050D000A9071092AA071092AB071092AC07109282
:1050E000A5071092A6071092A7071092A807109282
:1050F000B1071092B2071092B3071092B407109242
:10510000AD071092AE071092AF071092B007109241
:10511000BD071092BE071092BF071092C0071092F1
:10512000B5071092B6071092B7071092B807109201
:10513000B9071092BA071092BB071092BC071092E1
:10514000CD071092CE071092CF071092D007109281
:10515000DB070E94E03D6093C1077093C207809314
:10516000C3079093C4078AE290E00E94021660E0B1
:1051700076E081E091E00E944E156091C107709148
:10518000C2078091C3079091C4070E944E1560E04A
:1051900070E880E090E00E944E1580E060E170E0F1
:1051A0000E947F1500E011E0C80166E070E00E94F7
:1051B000671580E06AEC70E00E947F1563E673E596
:1051C00082E893E60E944E1581E095E30E943D152A
:1051D00081E00E9430158DE30E94301587E00E9427
:1051E000301581E00E943015C80166E070E00E9431
:1051F00067158FEF0E94301580E06FE270E00E942B
:105200007F158CE291E00E9474261F910F91089502
:105210000F931F93182F8093D807883129F08FEFB1
:105220009FEFAFEFBFEF08C08091AD079091AE0741
:10523000A091AF07B091B007809324049093250408
:10524000A0932604B0932704133051F00E94E03D50
:105250006093C1077093C2078093C3079093C407FC
:10526000E1E5F9E001900020E9F73197E155F940D7
:105270000E2F0F5F83E490E090932D0480932C0415
:1052800084E490E090932F0480932E048AE290E0CF
:105290000E94021660E076E081E091E00E944E15E7
:1052A0006091C1077091C2078091C3079091C407B4
:1052B0000E944E1580E090E00E943D15183119F0D3
:1052C00080E090E802C080E090E00E943D1560918F
:1052D000AD047091AE048091AF049091B0040E942F
:1052E0004E1580E06CE070E00E947F1580E091E058
:1052F00066E070E00E94671580E06AEC70E00E9452
:105300007F1563E673E582E893E60E944E1581E01F
:1053100095E30E943D1583E00E9430158CE00E94C9
:105320003015802F0E94301581E599E0602F70E0E4
:105330000E946715133019F582E30E94301584E04E
:105340000E943015809130049091310440960E9463
:10535000DD150E94FD140E944E1586E30E94301553
:1053600084E00E9430156091AD077091AE07809186
:10537000AF079091B0070E944E1519E115C0163184
:1053800011F015E211C082E30E94301584E00E9402
:1053900030156091A1077091A2078091A3079091A9
:1053A000A4070E944E151FE187E30E94301586E096
:1053B0000E94301581E00E94301583E00E94301574
:1053C00086E00E94301583E30E9430158AE30E9434
:1053D00030158BE30E9430158DE30E94301587E075
:1053E0000E94301581E00E94301580E091E066E077
:1053F00070E00E9467158FEF0E943015101B80E04F
:10540000612F70E00E947F158CE291E00E9474266B
:105410001F910F910895EF92FF920F931F93809128
:10542000D9079091DA07892B59F4A8E0B1E0EDE1B2
:10543000F1E082E101900D928150E1F760E0DCC083
:105440008091D807813031F0863121F0883111F018
:105450008931D9F5E090D507F090D60700E010E04B
:1054600088E091E06DE171E00E94EE3EE61AF70AF5
:10547000080B190BE092D107F092D2070093D307E3
:105480001093D4071E141F0410061106F4F0809127
:10549000D807813049F0863159F48091DB078F5F5E
:1054A0008093DB07833018F00E942A2803C086E12E
:1054B0000E940829682FA8E0B1E0EDE1F1E082E167
:1054C00001900D928150E1F701C060E0E090CD07BE
:1054D000F090CE070091CF071091D007D801C701F7
:1054E0000196A11DB11D0297A105B10508F484C064
:1054F0008091C5079091C607A091C707B091C807D2
:105500002091C9073091CA074091CB075091CC0731
:105510000097A105B10591F10197A109B109809307
:10552000C5079093C607A093C707B093C80721503B
:105530003040404050402093C9073093CA07409301
:10554000CB075093CC070894E108F1080109110931
:10555000E092CD07F092CE070093CF071093D007CB
:105560000097A105B10509F047C088E10E9408290C
:10557000682F882309F040C06CE03EC00894E10821
:10558000F10801091109211531054105510509F1FC
:10559000DA01C9010197A109B1098093C907909364
:1055A000CA07A093CB07B093CC07E092CD07F09247
:1055B000CE070093CF071093D0070097A105B10540
:1055C000D9F489E10E940829682F8823A9F46DE0A5
:1055D00013C0E092CD07F092CE070093CF0710934F
:1055E000D007E114F1040105110531F40E942A28C5
:1055F000682F882309F46EE0862F1F910F91FF908A
:10560000EF900895ACE1B0E0E8E0FBE20C94956225
:105610008091D807882309F4E8C1873109F4E5C1EE
:10562000809130049091310480519F4F0E94DD158C
:105630000E94DE14182F8F3F09F4C5C00E94DE14AB
:10564000082F153341F4813009F0D6C10E94DE14D1
:105650008093D707EDCF113071F4843009F0CCC1BD
:105660000E94FD146093A5077093A6078093A70777
:105670009093A807DDCF133071F4843008F4BCC1D7
:105680000E94FD146093A9077093AA078093AB074B
:105690009093AC071FC0163371F4843008F4ACC18A
:1056A0000E94FD146093AD077093AE078093AF071F
:1056B0009093B0070FC01630A1F4843008F49CC159
:1056C0000E94FD146093B1077093B2078093B307F3
:1056D0009093B407043009F4ABCF802F90E0049787
:1056E0006FC0133309F04BC0843009F0A1CF0E9482
:1056F000FD147B018C016093BD077093BE078093FE
:10570000BF079093C0078091B9079091BA07A09105
:10571000BB07B091BC070097A105B105B1F4C80162
:10572000B7012BE633E040E050E00E940D6228EE26
:1057300033E040E050E00E944C622093B907309380
:10574000BA074093BB075093BC078091B50790916F
:10575000B607A091B707B091B8070097A105B105AA
:1057600009F066CF16950795F794E794E092B50790
:10577000F092B6070093B7071093B80759CF1A33C2
:1057800071F4843009F054CF0E94FD146093B50782
:105790007093B6078093B7079093B80749CF1B3330
:1057A00071F4843009F044CF0E94FD146093B9076E
:1057B0007093BA078093BB079093BC0739CF90E0F2
:1057C0000E94211835CF80913004909131040496C5
:1057D0000E94DD158091D8079091D7078130B9F4E8
:1057E000923009F004C10E94FD142091C10730914C
:1057F000C2074091C3075091C4076217730784071B
:10580000950709F0F4C083E00E940829F1C09530A3
:1058100009F0D9C00E94FD142091C1073091C20740
:105820004091C3075091C407621773078407950717
:1058300009F0DDC087E18093D80780913004909112
:10584000310440960E94DD150E94FD14AB01BC019D
:105850004093AD045093AE046093AF047093B004D2
:1058600088E090E00E94CB638091A5079091A60705
:10587000A091A707B091A8078093B1049093B204B8
:10588000A093B304B093B4048091A9079091AA07A0
:10589000A091AB07B091AC078093B5049093B60488
:1058A000A093B704B093B8048091B1079091B20768
:1058B000A091B307B091B4078093610990936209F6
:1058C000A0936309B09364098091B5079091B607DE
:1058D000A091B707B091B8078093C5079093C6070A
:1058E000A093C707B093C8078091B9079091BA07F2
:1058F000A091BB07B091BC078093C9079093CA07DA
:10590000A093CB07B093CC078091BD079091BE07C1
:10591000A091BF07B091C0078093CD079093CE07A9
:10592000A093CF07B093D0078F5F9F4FAF4FBF4F6C
:1059300021F41092DA071092D907DE011196ECE1FA
:10594000F4E08CE101900D928150E1F76091AD049B
:105950007091AE048091AF049091B0040E94751EC6
:105960000E941C160E94C91A8C01A8950E943F2013
:10597000813019F40E941C1609C0823039F40E944B
:10598000A0278823B1F40E942A2813C00E94C91AB4
:10599000801B910B8D54914040F38091650981509B
:1059A000823030F481E090E090936D0980936C092F
:1059B00080E0ACE1B4E0FE0131969CE101900D92F3
:1059C0009150E1F715C0963091F40E94FD1420919A
:1059D000C1073091C2074091C3075091C4076217B5
:1059E00073078407950719F407C080E001C08FE0B2
:1059F0006C96E6E00C94B1620E942A28F9CFAF922F
:105A0000BF92DF92EF92FF920F931F93DF93CF939A
:105A10000F92CDB7DEB7F82EE92E9C0159018EE228
:105A2000D82E0E94DE14982F882331F40894A10800
:105A3000B108F501108219C0807C803C11F085010D
:105A40000AC00E94DE1411C099830E94DE14F8017E
:105A500081938F019981802F8A198917A8F3A90E44
:105A6000B11CF501D1925F01DCCF8F2D9E2D0F90DF
:105A7000CF91DF911F910F91FF90EF90DF90BF903A
:105A8000AF900895ACE4B0E0E8E4FDE20C948B62E2
:105A900080913004909131040E94DD15CE01019671
:105AA0006CE070E00E94191589819A810E94513E34
:105AB00020914609309147098217930709F06AC07F
:105AC0008D819E810E94513E6C01EE24FF243DE2B7
:105AD000A32EB12CAC0EBD1E2DE0822E912C8C0E6F
:105AE0009D1E14C0C5010E94FF2C0E94EB148C0166
:105AF0000E94EB140130110531F4019721F4C40127
:105B0000B5010E9469630894E11CF11CEC14FD04CA
:105B100048F38F8198850E94513E3C01EE24FF247A
:105B20009DE2492E512C4C0E5D1E31C0C2010E94D7
:105B3000FF2C0E94EB148C010E94EB144C010E947C
:105B4000FD145B016C010E94EB1401301105D1F4CE
:105B500021E082169104B1F48430910599F40E94F9
:105B6000FD14AB01BC01409348095093490960936F
:105B70004A0970934B09CE010D96960185010E944A
:105B8000683108C00E9421180894E11CF11CE61439
:105B9000F70460F280E0C45BDF4FE0E10C94A762A1
:105BA000AF92BF92DF92EF92FF920F931F93CF932A
:105BB000DF93182F092F8091610990916209A091BC
:105BC0006309B09164098093240490932504A09301
:105BD0002604B093270485E390E090932D048093EE
:105BE0002C0480E094E090932F0480932E040E9474
:105BF000E03D70934709609346098AE290E00E9475
:105C0000021680914609909147090E943D1580E057
:105C100091E00E943D1581E090E00E943D1580E0FA
:105C200090E00E943D1580E090E00E943D1580E0EC
:105C300090E00E943D15212F302FC901EC0140E179
:105C4000A42EB12C7E010E2D0C1BF701D080FEE29C
:105C5000DF1631F0DD2021F00894E11CF11CF3CFB8
:105C6000802F0E94301510E0CE01B8010E94671508
:105C70000F5F1F4FA00EB11EDD2019F0E701219626
:105C8000E1CF80E00E94301581E090E00E943D1558
:105C900081E090E00E943D15C50101960E947426A6
:105CA000DF91CF911F910F91FF90EF90DF90BF9008
:105CB000AF9008951F930E94DE14182F115412956F
:105CC000107F0E94DE1481548F70812B1F910895E4
:105CD0000F931F93CF93DF93EC0100E0899190E045
:105CE0000E94D462182F85958595859585958F5B43
:105CF0000E9430151F70812F8F5B0E9430150F5F3F
:105D0000003161F780E00E943015DF91CF911F9143
:105D10000F910895ACE1B0E0E0E9FEE20C948B62F3
:105D200080913004909131040E94DD15CE010196DE
:105D30006CE070E00E9419158B819C810E94513E9D
:105D40009C018F709070892B11F082E1EEC037FFBB
:105D50005AC089819A810E94513E20914609309112
:105D600047098217930709F0DFC08F8198850E9449
:105D7000513E019711F080E1D8C00E94DE148032BC
:105D800011F081E1D2C08E01035F1F4FC801902E38
:105D9000892E2DE1E22EF12CEC0EFD1E0E945A2ED2
:105DA000F80181938F01EE15FF05C1F71C8E0E944B
:105DB000DE140E94EB148C010E94EB147C010E9403
:105DC000FD145B016C010032110509F0ADC0F1E07A
:105DD000EF16F10409F0A8C00E94EB140E94EB1426
:105DE0000E94FD14AB01BC0140934809509349093E
:105DF00060934A0970934B09892D982D960185016E
:105E00000E94683191C020703877232B09F08CC034
:105E10008091320490913304C29709F085C0898142
:105E20009A810E94513E4C018D819E810E94513E7B
:105E30005C01CC24DD249DE0692E712C6C0E7D1E4E
:105E40008DE1482E512C4C0E5D1E31C00E94DE1497
:105E5000803209F069C083010E945A2EF8018193B3
:105E60008F01E415F505C1F71C8E0E94DE140E9417
:105E7000EB147C010E94EB140197B1F4F0E2EF16F1
:105E8000F10451F4C30161E579E00E946063009779
:105E900059F400E015E84FC081E2E816F10421F45E
:105EA0008D858A3209F445C00894C11CD11CCA14DE
:105EB000DB0460F239C086E090E00E943D1580E08E
:105EC00090E00E943D156091AD047091AE04809108
:105ED000AF049091B0040E944E158EE390E021C073
:105EE0008DE390E00E943D1581E00E94301581E530
:105EF00099E06FE070E00E94671580E00E94301525
:105F000080E094E00E943D1580E091E066E070E062
:105F10000E94671580E064E270E00E947F1585E7CB
:105F200090E00E94742601C080E06C96E0E10C9441
:105F3000A76200E014E88AE290E00E940216C40121
:105F40000E943D15C8010E943D1580E090E00E942E
:105F50003D1581E090E00E943D1580E090E00E94B8
:105F60003D1580E090E00E943D1580E20E943015D2
:105F7000CE010D960E94682EC7010E943D1581E05A
:105F800090E00E943D1568E572E080E090E00E949C
:105F90004E15E0E2EE16F10409F0A2CF8CCF0F937C
:105FA0001F938C018091B1049091B204A091B3042D
:105FB000B091B40480959095A095B0952091AD04D2
:105FC0003091AE044091AF045091B004822B932BDA
:105FD000A42BB52B8093240490932504A09326042E
:105FE000B093270489E890E090932D0480932C04CB
:105FF00090932F0480932E040E94E03D70934709F4
:10600000609346098AE290E00E9402168091460958
:10601000909147090E943D1580E191E00E943D1555
:1060200081E090E00E943D1580E090E00E943D15E7
:1060300080E090E00E943D1580E090E00E943D15D8
:1060400080E20E943015C8010E94682E80E290E034
:106050000E943D1581E090E00E943D1582E390E0B2
:106060000E9474261F910F910895E0E2F8E0848168
:106070008130A1F480819181A281B3810097A10533
:10608000B10561F00197A109B10980839183A283D1
:10609000B3830097A105B10509F41482B99689E08C
:1060A000E836F80721F70895A9E2B0E0EAE5F0E361
:1060B0000C9493627C010CEF17E06E010894C11CF4
:1060C000D11CD601F80189E201900D928150E1F7CF
:1060D00089A5813059F4C601B7010E946063009719
:1060E00029F429A13AA14BA15CA10AC0075D1F4F69
:1060F00089E00434180729F720E030E040E050E060
:10610000B901CA01A996E8E00C94AF62CF93DF937E
:1061100080914E09813001F5CCEDD7E0CE0168E4E5
:1061200079E00E945B3E813009F4C3C0FE0101901A
:106130000020E9F73197EC1BFD0B709738F4CE0186
:106140006EE270E00E945563009711F084E001C098
:1061500082E080934E09A9C0823009F58CED97E06A
:106160000E945430609348097093490980934A090A
:1061700090934B09611571058105910509F099C04E
:106180000E94C91A90934509809344098CED97E0C9
:106190000E94CF2F282F10924D0983E053C08330E7
:1061A00079F58091480990914909A0914A09B091E7
:1061B0004B090097A105B10509F07BC00E94C91ADF
:1061C0002091440930914509821B930B885E9340CE
:1061D00008F46BC080914D098F5F80934D09833027
:1061E00020F0209174072D5E61C00E94C91A90931F
:1061F0004509809344098CED97E00E94CF2F53C04E
:10620000843019F58CED97E00E9454306093480972
:106210007093490980934A0990934B096115710560
:106220008105910509F045C00E94C91A909345095E
:10623000809344098CED97E00E94D02D282F109276
:106240004D0985E080934E0931C0853071F580910C
:10625000480990914909A0914A09B0914B090097CA
:10626000A105B10531F50E94C91A20914409309168
:106270004509821B930B885E9340B8F080914D09CD
:106280008F5F80934D09833020F020917407295E41
:106290000DC00E94C91A90934509809344098CED62
:1062A00097E00E94D02D282F01C020E080E090E0F0
:1062B00003C020E081E090E09093500980934F0963
:1062C000019711F410924E09822FDF91CF9108951A
:1062D000A0E0B0E0EEE6F1E30C948D62EC016A011F
:1062E0007B014801590100E010E089E2682E712C21
:1062F000069DC001079D900D169D900D11248450A0
:10630000984FBE010E946063009739F10F5F1F4FE5
:106310000830110569F720914C09822F8F5F877033
:1063200080934C0930E089E290E0289F8001299F0A
:10633000100D389F100D11240450184FC801BE01D4
:106340000E946963F801C0A2D1A2E2A2F3A284A2D2
:1063500095A2A6A2B7A281E080A7CDB7DEB7EEE0F6
:106360000C94A962A8E0B0E0E8EBF1E30C94916230
:106370006D837E838F83988719821A821B821C8289
:1063800029813A814B815C81F8EEAF2EE3E0BE2E8D
:10639000CC24DD24EE24FF2400E010E00E94985B72
:1063A000952FB901842F2896EAE00C94AD62A4E2FF
:1063B000B0E0EDEDF1E30C9493621091740710934B
:1063C000750700E0B5E0EB2EF12CEC0EFD1E6E0122
:1063D0000894C11CD11C1F5F1370E12FF0E0EE0F79
:1063E000FF1FEC5AFE4F65917491C7010E946963CB
:1063F000C701B6010E945B3E813041F489819A81D8
:10640000AB81BC810097A105B10519F01093740709
:1064100003C00F5F0430F9F6A496E8E00C94AF6275
:10642000AF92BF92CF92DF92EF92FF920F931F93A2
:10643000609324047093250480932604909327048A
:106440008BE790E090932D0480932C0490932F047D
:1064500080932E048AE290E00E94021683E20E945A
:10646000301580E067E270E00E947F15F894E090BC
:10647000820BF090830B0091840B1091850B60913F
:10648000800B7091810B882777FD8095982F0E9453
:10649000B2315B016C017894609386077093870733
:1064A000809388079093890780E89EE7AAEAB3E87B
:1064B000E80EF91E0A1F1B1FC801B7010E944E15E6
:1064C000C601B5010E944E1580E390E00E9474263B
:1064D0001F910F91FF90EF90DF90CF90BF90AF9002
:1064E00008951F9310917609112309F480C011308B
:1064F000A1F480917407E82FF0E0EE0FFF1FEC5A33
:10650000FE4F659174918CED97E00E946963109342
:106510004E0982E0809376096AC0123089F5809135
:106520004F0990915009019709F061C010925009EC
:1065300010924F09609148097091490980914A0968
:1065400090914B096093F0067093F1068093F206E8
:106550009093F30610929E070E941032182F882302
:1065600051F483E0809376090E94C91A90939707AB
:106570008093960702C0109276090E94D73138C0E6
:106580001330A9F50E94C91A2091960730919707F8
:10659000821B930B209198073091990782179307DC
:1065A00030F180919E078F5F80939E07833040F08B
:1065B00010937D0110917507145E0E949D0B18C009
:1065C0006091F0067091F1068091F2069091F306C9
:1065D0000E941032182F882339F40E94C91A909310
:1065E00097078093960704C01092760901C010E0C7
:1065F000812F1F910895809167098770823019F467
:1066000084EF90E004C0833041F480EF90E00E947A
:10661000341880E00E94301508956091AD047091A7
:10662000AE048091AF049091B0040E944E1508957D
:10663000AF92BF92CF92DF92EF92FF920F931F9390
:1066400080917A0790917B07A0917C07B0917D079C
:106650008093240490932504A0932604B0932704E8
:106660008BE790E090932D0480932C0490932F045B
:1066700080932E048091770990917809892B19F4E1
:1066800005EE10E102C005E211E08AE290E00E940E
:106690000216802F0E943015812F0E9430156091C4
:1066A0009A0770919B0720E030E84FE0C9018623EC
:1066B0009723892B29F4415019F036952795F6CF69
:1066C000842F0E94301586EF0E94301560917E075E
:1066D00070917F0780918007909181070E944E15ED
:1066E000609182077091830780918407909185075C
:1066F0000E944E150E94FB3260919407709195079D
:1067000080E090E00E94B2317B018C0160918E07A5
:1067100070918F0780919007909191076058714810
:1067200085459C470E944E15C801B7010E944E1531
:1067300080E060E170E00E947F15F894E090820BA9
:10674000F090830B0091840B1091850B6091800B6E
:106750007091810B882777FD8095982F0E94B23128
:106760005B016C01789480E89EE7AAEAB3E8E80E42
:10677000F91E0A1F1B1FC801B7010E944E15C60152
:10678000B5010E944E1580E390E00E9474261F918F
:106790000F91FF90EF90DF90CF90BF90AF90089552
:1067A000ABE6B0E0E6EDF3E30C948962809130044F
:1067B000909131040E94DD15CE01819660E370E076
:1067C0000E94191599A1892F8770843009F01CC483
:1067D00080917609882309F4ADC7892F807C809346
:1067E00006019AA1803C21F0992311F0903158F0D4
:1067F00082E080937D0110924E09109276090E94EA
:106800009D0B8BE198C79F5F909307016DA17EA1BF
:106810008FA198A50E94553E60937E0770937F07D5
:10682000809380079093810769A57AA58BA59CA585
:106830000E94553E6093820770938307809384077C
:1068400090938507FE01E05CFF4F90812FAD5EAD18
:106850006DAD7CADABADDAAC99ACFE01EC5BFF4F3E
:10686000C080FE01ED5BFF4FB080FE01EE5BFF4F8D
:10687000A080FE01EF5BFF4F7080FE01E85BFF4FE1
:106880008081FE01E95BFF4F3081FE01EA5BFF4F33
:106890004081FE01EB5BFF4FE081E82EE91A91E0B9
:1068A0008E1508F090E0832F821B21E0381708F046
:1068B00020E0F82EF91A91E08F1508F090E0292BCE
:1068C000842F851B31E0481708F030E0082F021BA9
:1068D00091E0801708F090E0392B8E2F861B21E085
:1068E000E81708F020E0182F131B91E0811708F03B
:1068F00090E0292B8C2D871B31E0C81608F030E082
:10690000B82FB21B91E08B1708F090E0392B8B2D3C
:106910008A1B21E0B81608F020E0A82FA31B91E005
:106920008A1708F090E0292B8A2D8D1991E0A8167E
:1069300008F090E0F82FF21B21E08F1708F020E01C
:10694000922BE72DE919E91B9701A8016B2F7A2FEC
:106950008F2F9E2F52F52E2D2F5F81E02E1508F0E0
:1069600080E0382F3F0D81E03F1508F080E0482F90
:10697000400F81E0401708F080E0582F510F81E070
:10698000511708F080E0682F6B0F81E06B1708F05B
:1069900080E0782F7A0F81E07A1708F080E08F0F7F
:1069A00091E08F1708F090E09E0F01E00E94135BCA
:1069B000622E532E442E352E262E66967FAF669776
:1069C00067968FAF679768969FAF6897FE01E45B05
:1069D000FF4FC080FE01E55BFF4FB080FE01E65B2C
:1069E000FF4FA080FE01E75BFF4F7080FE01E05B80
:1069F000FF4F0081FE01E15BFF4FF080FE01E25B93
:106A0000FF4F9080FE01E35BFF4F808080918A07FB
:106A100090918B07A0918C07B0918D078058914879
:106A2000A545BC47182F8D8B9E8BAF8BB88F60917F
:106A300092077091930780E090E00E94B231698BD9
:106A40007A8B8B8B9C8B872F3B89492F5E897F8923
:106A5000E88DD02ED61A91E00D1508F090E02F2D7C
:106A6000281B822F21E0F81608F020E0E82EE91A12
:106A700091E08E1508F090E0292B892D831B31E0E1
:106A8000981608F030E0F82EF21A91E08F1508F011
:106A900090E0392B882D841B21E0881608F020E037
:106AA000082F031B91E0801708F090E0292B3C2D64
:106AB000311B132F91E0C31608F090E0B12FB21BE9
:106AC00081E01B1708F080E0982B8B2D851B21E0BF
:106AD000B81608F020E0A82FA91B91E08A1708F04B
:106AE00090E0292B8A2D871B91E0A81608F090E0F2
:106AF000F82FF21B21E08F1708F020E0922B7E1A6E
:106B0000E72DE91B2D2D3E2D4F2D502F6B2F7A2F6A
:106B10008F2F9E2F52F52D2D2F5F81E02D1508F020
:106B200080E0382F3E0D81E03E1508F080E0482FD0
:106B30004F0D81E04F1508F080E0582F500F81E095
:106B4000501708F080E0682F6B0F81E06B1708F09A
:106B500080E0782F7A0F81E07A1708F080E08F0FBD
:106B600091E08F1708F090E09E0F01E00E94135B08
:106B7000A32FB42F152F062FF72ED82EC22EC60CFA
:106B8000F1E0C21608F0F0E03A2F350DE1E03A17D7
:106B900008F0E0E0EF2EE30E21E0E31608F020E03D
:106BA000E22B4B2F440D31E04B1708F030E0AE2FB5
:106BB000A40F21E0A41708F020E0322B512F530D31
:106BC00041E0511708F040E0F32FF50F21E0F517F1
:106BD00008F020E0422B602F620D31E0601708F0D2
:106BE00030E0E42FE60F21E0E61708F020E0322B3A
:106BF00066967FAD66977F0D41E07F1508F040E017
:106C0000532F570F21E0571708F020E0422B6796CB
:106C10008FAD67978D0D21E08D1508F020E0480FAE
:106C200031E0481708F030E0232B68968FAD689765
:106C3000980F290FC98AEA8AAB8BFC8BED8B5E8B90
:106C40004F8B288F4D885E886F88788C89899A89C8
:106C5000AB89BC894C015D01CC24DD2476019C010B
:106C6000A50160E070E080E090E002E00E94945AAC
:106C7000122F232E69964FAF69976A965FAF6A9776
:106C80006B966FAF6B976C967FAF6C976D968FAF6F
:106C90006D976E969FAF6E9705E00E94945AA32F52
:106CA000B42F052F6F966FAF6F97A0967FAFA09709
:106CB000A1968FAFA197A2969FAFA297322E311ABD
:106CC000F1E0231508F0F0E03A2F3219E1E0A317C4
:106CD00008F0E0E0132F1F1B21E0311708F020E03F
:106CE000E22B4B2F69969FAD6997491B31E0B41792
:106CF00008F030E0B42FBE1B21E04B1708F020E075
:106D0000322B502F6A96AFAD6A975A1B41E0051798
:106D100008F040E0052F031B21E0501708F020E0A9
:106D2000422B6F966FAD6F976B96EFAD6B976E1BA7
:106D300031E06F96FFAD6F97F61708F030E0962FB1
:106D4000941B21E0691708F020E0322BA0967FAD5C
:106D5000A0976C962FAD6C97721B41E0A0968FADFB
:106D6000A097871708F040E0A72FA31B21E07A1710
:106D700008F020E0422BA1968FADA1976D96EFAD64
:106D80006D978E1B21E0A196FFADA197F81708F033
:106D900020E0E82FE41B31E08E1708F030E0232BD1
:106DA000A296FFADA2976E963FAD6E97F31BF21BB6
:106DB000232C280C31E0231408F030E0812F890DBA
:106DC00041E0811708F040E0380F51E0381708F033
:106DD00050E0452B8B2F8A0D51E08B1708F050E0C7
:106DE000480F61E0481708F060E0562B202F2B0D6C
:106DF00081E0201708F080E0520F61E0521708F0A0
:106E000060E0682B690F71E0691708F070E07A0F95
:106E100081E07A1708F080E08E0F91E08E1708F07D
:106E200090E0222D9F0F03E00E94945A298F3A8F01
:106E30004B8F5C8F6D8F7E8F8F8F98A3ED8CFE8C28
:106E40000F8D18A180911B0190911C01892BC9F411
:106E500080919F079091A007009799F0A30192015C
:106E600077FE07C022273327A901241935094609CF
:106E70005709A0E0B0E082179307A407B5070CF408
:106E800059C48701F8948091820B9091830BA09153
:106E9000840BB091850B840D951DA61DB71D8093A5
:106EA000820B9093830BA093840BB093850B8091FE
:106EB000800B9091810B8E0D9F1D9093810B809381
:106EC000800B8091800B9091810B97FF2AC080915D
:106ED000820B9091830BA091840BB091850B1816B7
:106EE00019061A061B06ECF48091820B9091830B15
:106EF000A091840BB091850B0197A109B1098093F2
:106F0000820B9093830BA093840BB093850B80919D
:106F1000800B9091810B88519C4F9093810B8093B3
:106F2000800B8091820B9091830BA091840BB09188
:106F3000850B80938E0790938F07A0939007B09353
:106F400091078091800B9091810B9093950780938E
:106F50009407789477FE0AC0101611063CF4089442
:106F6000411C511C611C711C085E1340D301C201FD
:106F700080509048AF4FBF4F80509040A140B040EC
:106F800038F08FEF9FE7909377078093760704C0E0
:106F9000509277074092760710937907009378070D
:106FA00080917F09882361F1C301B20128EE33E0AB
:106FB00040E050E00E940D629B01AC01C801AA278D
:106FC00097FDA095BA2F820F931FA41FB51FB7FD81
:106FD00004C0B801620F731F0AC0C301B20128E1E7
:106FE0003CEF4FEF5FEF0E940D62601B710B7093DF
:106FF0007E0960937D096D54714014F081E001C0F9
:1070000082E080937F0990C3833009F0E9C0292F83
:10701000287380917709909178090197F1F5509044
:107020000601522A40900701E0908E07F0908F07EA
:10703000009190071091910780E89EE7AAEAB3E8D3
:10704000E80EF91E0A1F1B1F6091940770919507A7
:1070500080E090E00E94B2313B014C01A0908A0791
:10706000B0908B07C0908C07D0908D0780E89EE78A
:10707000AAEAB3E8A80EB91ECA1EDB1E60919207E9
:107080007091930780E090E00E94B23165966CAFFA
:107090007DAF8EAF9FAF659713C030EC532E522A51
:1070A00065961CAE1DAE1EAE1FAE65976624772496
:1070B0004301AA24BB246501EE24FF248701442454
:1070C0008AE290E00E940216852D84600E943015AD
:1070D000842D0E9430158BA10E94301586EF0E94EE
:1070E000301560E070E080E090E00E944E1560E0B6
:1070F00070E080E090E00E944E150E94FB32C801D3
:10710000B7010E944E15C401B3010E944E15809133
:10711000770990917809019799F4CE0181968C01B5
:10712000085D1F4F20E3E22EF12CE80EF91ED80176
:107130008D918D010E9430150E151F05C1F70CC0F1
:1071400060E070E080E090E00E944E1560E070E04A
:1071500080E090E00E944E15C601B5010E944E15D8
:1071600065966CAD7DAD8EAD9FAD65970E944E1559
:107170008091770990917809019739F0AA24BB246E
:107180006501EE24FF2487011EC0F894E090820B75
:10719000F090830B0091840B1091850B80E89EE7A3
:1071A000AAEAB3E8E80EF91E0A1F1B1F6091800BC4
:1071B0007091810B882777FD8095982F0E94B231BE
:1071C0005B016C017894C801B7010E944E15C6019D
:1071D000B5010E944E1580E390E00E947426ABC278
:1071E000853009F0A7C2809167098770813009F066
:1071F000A1C2892F807C809306019AA1803C09F46A
:1072000099C2992309F496C2903109F493C29F5F01
:10721000909307016DA17EA18FA198A50E94553E74
:1072200060937E0770937F07809380079093810718
:1072300069A57AA58BA59CA50E94553E60938207FF
:10724000709383078093840790938507FE01E05B2A
:10725000FF4FD080FE01E15BFF4FC080FE01E25B8B
:10726000FF4FA080FE01E35BFF4F10813D2DD982CF
:107270002C2DCA829A2DAB82812F1C83FE01E45BE8
:10728000FF4FD080FE01E55BFF4FC080FE01E65B53
:10729000FF4FA080FE01E75BFF4F1081DD82CE82B1
:1072A000AF821887032FF22EE92EB82E832F822B60
:1072B000892B8B298D298C298A29812B09F43AC2A3
:1072C000F8948091820B9091830BA091840BB091E4
:1072D000850B80589148A545BC478D839E83AF831D
:1072E000B8876091800B7091810B882777FD80951E
:1072F000982F0E94B23169837A838B839C83789420
:1073000089812A813B814C815D81AE81BF819884D6
:10731000F02FF81B91E00F1708F090E08F2D821BE3
:1073200021E0F81608F020E0E82FE91B91E08E1725
:1073300008F090E0292B8E2D831B31E0E81608F031
:1073400030E0782F721B91E0871708F090E0392B1E
:107350008B2D841B21E0B81608F020E0682F631BFA
:1073600091E0861708F090E0292B8D2D851B31E0E8
:10737000D81608F030E0582F521B91E0851708F01E
:1073800090E0392B8C2D8A1B21E0C81608F020E0F4
:10739000482F431B91E0841708F090E0292B8A2D99
:1073A0008B1B91E0A81608F090E0382F321B21E0EB
:1073B000831708F020E0922B1919191BF983EA832F
:1073C0007B836C835D834E833F8318874D805E8013
:1073D0006F80788489819A81AB81BC814C015D0189
:1073E000CC24DD2476019C01A50160E070E080E002
:1073F00090E002E00E94945A122F232EA3964FAFE2
:10740000A397A4965FAFA497A5966FAFA597A696EE
:107410007FAFA697A7968FAFA797A8969FAFA8977D
:1074200005E00E94945AA32FB42F052FA9966FAFA1
:10743000A997AA967FAFAA97AB968FAFAB97AC965A
:107440009FAFAC97322E311AF1E0231508F0F0E02F
:107450003A2F3219E1E0A31708F0E0E0132F1F1BC9
:1074600021E0311708F020E0E22B4B2FA3969FADCF
:10747000A397491B31E0B41708F030E0B42FBE1BCE
:1074800021E04B1708F020E0322B502FA496AFAD2F
:10749000A4975A1B41E0051708F040E0052F031B95
:1074A00021E0501708F020E0422BA9966FADA99774
:1074B000A596EFADA5976E1B31E0A996FFADA997F4
:1074C000F61708F030E0962F941B21E0691708F0BA
:1074D00020E0322BAA967FADAA97A6962FADA6974D
:1074E000721B41E0AA968FADAA97871708F040E07B
:1074F000A72FA31B21E07A1708F020E0422BAB96C0
:107500008FADAB97A796EFADA7978E1B21E0AB96FB
:10751000FFADAB97F81708F020E0E82FE41B31E04F
:107520008E1708F030E0232BAC96FFADAC97A896F1
:107530003FADA897F31BF21B232C280C31E023143A
:1075400008F030E0812F890D41E0811708F040E01C
:10755000380F51E0381708F050E0452B8B2F8A0D7B
:1075600051E08B1708F050E0480F61E0481708F031
:1075700060E0562B202F2B0D81E0201708F080E0D3
:10758000520F61E0521708F060E0682B690F71E05C
:10759000691708F070E07A0F81E07A1708F080E050
:1075A0008E0F91E08E1708F090E0222D9F0F03E0E0
:1075B0000E94945A29873A874B875C876D877E871C
:1075C0008F87988BED84FE840F85188980911B012D
:1075D00090911C01892BC9F480919F079091A0077D
:1075E000009799F0A301920177FE07C02227332765
:1075F000A9012419350946095709A0E0B0E082170E
:107600009307A407B5070CF495C09701F8948091EF
:10761000820B9091830BA091840BB091850B840D0C
:10762000951DA61DB71D8093820B9093830BA0938D
:10763000840BB093850B8091800B9091810B8E0D04
:107640009F1D9093810B8093800B8091800B909174
:10765000810B97FF2AC08091820B9091830BA091A0
:10766000840BB091850B181619061A061B06ECF44C
:107670008091820B9091830BA091840BB091850B2C
:107680000197A109B1098093820B9093830BA0937A
:10769000840BB093850B8091800B9091810B885166
:1076A0009C4F9093810B8093800B8091820B9091E3
:1076B000830BA091840BB091850B80938E079093E0
:1076C0008F07A0939007B09391078091800B9091C2
:1076D000810B9093950780939407789477FE0AC066
:1076E000121613063CF40894411C511C611C711CB9
:1076F000285E3340D301C20180509048AF4FBF4F46
:1077000080509040A140B04038F08FEF9FE79093B9
:1077100077078093760704C05092770740927607E8
:10772000309379072093780781E090E09093890B5C
:107730008093880B80E0C559DF4FE2E10C94A5628D
:107740008091770990917809892B11F480E0089550
:107750008AE290E00E940216F8946091820B709188
:10776000830B8091840B9091850B789460587148BD
:1077700085459C470E944E1584E090E00E94742647
:107780000895DB01982F92959F702CE531E0F90167
:10779000E90FF11DE491EC938F70280F311DF90171
:1077A000849111968C93119712961C921297CB018B
:1077B0000895DB01292F22952F704CE551E0FA0145
:1077C000E20FF11DE491EC939F70FA01E90FF11DB6
:1077D000E4911196EC931197982F92959F70FA016E
:1077E000E90FF11DE4911296EC9312978F70480FF8
:1077F000511DFA01849113968C93139714961C9241
:107800001497CB010895DA01292F22952F704CE5AA
:1078100051E0FA01E20FF11DE491EC939F70FA013F
:10782000E90FF11DE4911196EC931197982F929521
:107830009F70FA01E90FF11DE4911296EC931297F3
:107840008F70FA01E80FF11DE4911396EC931397F2
:10785000872F82958F70FA01E80FF11DE49114963D
:10786000EC9314977F70FA01E70FF11DE4911596E0
:10787000EC931597862F82958F70FA01E80FF11D12
:10788000E4911696EC9316976F70460F511DFA010E
:10789000849117968C93179718961C921897CD0180
:1078A0000895282FDB0164E60E942C62392F822F75
:1078B0000E942C62805DFD018193832F6AE00E940B
:1078C0002C62805D11968C931197832F0E942C62FD
:1078D000905D91831282CD010895A0E0B0E0E3E7CE
:1078E000FCE30C949462482FF92EE62ED72E862FB7
:1078F000972F9C01E901E0E1F7E200E010E0842F1E
:107900009F2DBF010E943862262F842F9F2DBF011B
:107910000E943862482FF92E205D2993CF016AE03A
:1079200070E00E943862FB010F5F1F4F04301105A9
:1079300031F7405D488319828E2D9D2DCDB7DEB77E
:10794000E7E00C94B062A0E0B0E0E9EAFCE30C945C
:107950008C62062F772E4C01642E552E842F952F86
:107960009C01E901C12C8AECD82E8AE9E82E8BE330
:10797000F82EAA24BB24602F772DC401A7019601FD
:107980000E944C62122F602F772DC401A70196012F
:107990000E944C62062F772E4C01105D1993C7018F
:1079A000B6012AE030E040E050E00E944C62C9019C
:1079B000DA016C017D010894A11CB11C89E0A816B4
:1079C000B104C9F6005D08831982862D952DCDB7C7
:1079D000DEB7EFE00C94A862EF92FF920F931F9333
:1079E0008B019C01F42EE52E97FD04C0842F952F6A
:1079F000FC010CC030952095109501951F4F2F4F1D
:107A00003F4F842F952FFC018DE28193C901B8016E
:107A1000AF010E94A33C8F2D9E2D1F910F91FF90CF
:107A2000EF9008951F93CF93DF93EC0120E030E0B7
:107A300040E050E01881812F80538A30C8F4CA0199
:107A4000B9012AE030E040E050E00E940D629B0165
:107A5000AC01812F992787FD9095C097AA2797FDA4
:107A6000A095BA2F280F391F4A1F5B1F2196E2CF1E
:107A7000203080E0380781E0480780E0580720F098
:107A80002FEF3FEF40E050E0C901DF91CF911F9110
:107A90000895982F8154863010F487E307C0892F0A
:107AA0008156863010F487E501C080E3981B892F4A
:107AB0000895FF920F931F938C01FC0180810E9417
:107AC000493DF82EF29490EFF922F80181810E944D
:107AD000493D8F708F291F910F91FF900895EF926C
:107AE000FF920F931F938C01FC0180810E94493DFE
:107AF000F82EF29430EFF322F80181810E94493D83
:107B00008F70F82AF80182810E94493DE82EE294A4
:107B100020EFE222F80183810E94493D8F708E2977
:107B20009F2D1F910F91FF90EF900895CF92DF92BC
:107B3000EF92FF920F931F938C01FC0180810E94B2
:107B4000493DC82EC29470EFC722F80181810E947E
:107B5000493D8F70C82AF80182810E94493DD82E84
:107B6000D29460EFD622F80183810E94493D8F7044
:107B7000D82AF80184810E94493DF82EF29450EFF2
:107B8000F522F80185810E94493D8F70F82AF8019D
:107B900086810E94493DE82EE29440EFE422F801FC
:107BA00087810E94493D8F708E29682F7F2D8D2DF2
:107BB0009C2D1F910F91FF90EF90DF90CF90089533
:107BC000EF92FF920F931F9380917E0190917F011E
:107BD000A0918001B09181017C018D012BE0EE0C20
:107BE000FF1C001F111F2A95D1F7E826F9260A2746
:107BF0001B278091820190918301A0918401B09113
:107C0000850180937E0190937F01A0938001B093C2
:107C100081018091860190918701A0918801B091A6
:107C200089018093820190938301A0938401B09392
:107C3000850180918A0190918B01A0918C01B09176
:107C40008D018093860190938701A0938801B09362
:107C500089019C01AD01F3E156954795379527952C
:107C6000FA95D1F7282739274A275B272E253F2564
:107C700040275127EF2CF02E012F11272E253F25CD
:107C80004027512720938A0130938B0140938C0128
:107C900050938D01B901CA011F910F91FF90EF9090
:107CA0000895282F892F922F0895362F272F692F77
:107CB000782FC9010895A0E2B0E0E1E6FEE30C945C
:107CC0008F629C015B018E010F5F1F4FC801B901DC
:107CD0000E946963CC24DD247601980140E1842E62
:107CE000912C8C0E9D1EF80180818E3291F41082B1
:107CF000C9010E94123DA0E0B0E08C299D29AE2967
:107D0000BF29CC24D82EE92EFA2E98012F5F3F4FA1
:107D10002BC08823E9F4CE0101960817190731F426
:107D2000F501108211821282138210C0F8011082B4
:107D3000C9010E94123DA0E0B0E08C299D29AE2926
:107D4000BF29F50180839183A283B38381E013C0AF
:107D5000992787FD9095C0970A9730F0F50110821A
:107D600011821282138206C00815190519F00F5FDF
:107D70001F4FB9CF80E0A096ECE00C94AB62CF929D
:107D8000DF92EF92FF920F931F936B01E82E8A010F
:107D9000892FBA010E94513C5EE2F52EF801F38270
:107DA000B8016C5F7F4F8E2D0E94513CF801F78225
:107DB000B801685F7F4F8D2D0E94513CF801F3861A
:107DC000B801645F7F4F8C2D0E94513CC8011F9108
:107DD0000F91FF90EF90DF90CF900895CF92DF92B8
:107DE000EF92FF920F931F936B010E94B11D7B01D5
:107DF0008C01C6010E94B11D9B01AC012E193F09E7
:107E0000400B510BB901CA011F910F91FF90EF90E8
:107E1000DF90CF900895A4E0B0E0E1E1FFE30C949F
:107E20009762162F072F0E94B11D20917701309184
:107E300078014091790150917A01260F371F481F30
:107E4000591F29833A834B835C83CE0101960E949C
:107E5000091EAC01009711F480E00BC0812F902F18
:107E60009C01D901FA0182E101900D928150E1F764
:107E700081E02496E4E00C94B362A4E0B0E0E3E493
:107E8000FFE30C949362D62EC72E79018A010E94DB
:107E9000B11D6E197F09800B910B69837A838B83E7
:107EA0009C83CE0101960E94091EAC01009711F43B
:107EB00080E00BC08D2D9C2D9C01D901FA0182E13F
:107EC00001900D928150E1F781E02496E8E00C9456
:107ED000AF62EF92FF920F931F93E82EF62E8A0166
:107EE000FA940E94941BF8018083813131F48E2D25
:107EF0008F5FF81660F480E00AC0823111F08E2D99
:107F000006C0EE2011F48F2D02C08E2D81501F91DE
:107F10000F91FF90EF900895A0E0B0E0E2E9FFE359
:107F20000C948A62C82E362E7A01B22EE8010E9485
:107F3000311AEB2DFF27E7FDF095EE0DFF1D1082A6
:107F4000F7019081892F80538A3010F4182F08C0D0
:107F5000892F8154863010F010E002C0192F17537A
:107F6000A8951B9BFDCF81E00E94E419219711F099
:107F70008AE001C080E1012F112707FD1095DC2C5C
:107F8000C0E0D0E04B2C552447FC5094882E992417
:107F900087FC909434010894610871085701AC0E75
:107FA000BD1E8D2D632D0E94F8190A30110518F49D
:107FB000802F805D02C0802F895C0E94C8190E94BA
:107FC000DC190E94941B813141F40F5F1F4F08158B
:107FD00019054CF000E010E006C0823179F4015040
:107FE000104017FD83010A30110518F4802F805DC1
:107FF00002C0802F895CF5018083D0CF833151F599
:108000002196D394F701EC0FFD1F8081992787FDFE
:1080100090950E94C062892B11F42196D394C415C7
:10802000D5051CF0DC2CC0E0D0E0F701EC0FFD1F03
:10803000E0818E2F80538A3040F08E2F815486301D
:1080400010F080E002C08E2F8753082F112707FD04
:108050001095A4CF843119F401E010E005C08931F6
:1080600009F09CCF00E010E080E00E94E419C80114
:10807000CDB7DEB7E1E10C94A6628091940B81301C
:10808000C1F580918E0B90918F0BA091900BB091C8
:10809000910B0196A11DB11D80938E0B90938F0BB8
:1080A000A093900BB093910B80918E0B90918F0BBE
:1080B000A091900BB091910B80938E0790938F07B6
:1080C000A0939007B09391078093820B9093830BBA
:1080D000A093840BB093850B109295071092940790
:1080E00081E090E09093890B8093880B1092940B21
:1080F0003EC08091920B823099F08091820B9091DA
:10810000830BA091840BB091850B0196A11DB11D2D
:108110008093820B9093830BA093840BB093850B79
:10812000809167098770823031F52091680930911C
:10813000690921153105D9F080918C0B90918D0B37
:10814000019690938D0B80938C0B80918C0B90916A
:108150008D0B8217930778F089E080937D018091E1
:108160007C01843041F083E080937C0104C0109254
:108170008D0B10928C0B80917C018130C1F4809129
:108180006A0990916B09892B91F080918A0B9091EB
:108190008B0B019790938B0B80938A0B80918A0BAA
:1081A00090918B0B892B19F482E080937C0181E004
:1081B00090E09093870B8093860B08951F920F9207
:1081C0000FB60F9211242F933F934F935F936F93AA
:1081D0007F938F939F93AF93BF93EF93FF9382E02F
:1081E00083BD1092B2001CBA1DBA88EC80937B014B
:1081F0008091940B8230C1F41092810B1092800B0D
:10820000109295071092940781E090E09093890B6B
:108210008093880B10928D0B10928C0B1092940B04
:108220009093870B8093860B8091940B813091F40F
:10823000809167098770833039F484E690E09093E9
:10824000810B8093800B04C01092810B1092800BE5
:108250000E943D408AE08093930BFF91EF91BF9184
:10826000AF919F918F917F916F915F914F913F91CE
:108270002F910F900FBE0F901F9018951F920F9285
:108280000FB60F9211240F900FBE0F901F901895EC
:108290001F920F920FB60F9211240F900FBE0F90E6
:1082A0001F9018951F920F920FB60F9211242F93C3
:1082B0003F934F935F936F937F938F939F93AF936E
:1082C000BF93EF93FF938091800B9091810B019668
:1082D0009093810B8093800B8091940B8230C9F432
:1082E0001092810B1092800B1092950710929407B8
:1082F00081E090E09093890B8093880B10928D0B16
:1083000010928C0B1092940B9093870B8093860B9A
:108310000DC08091800B9091810B885E9340BCF0E2
:108320001092810B1092800B0E943D408091930B24
:10833000882331F08091930B81508093930B07C079
:1083400080917D01873019F486E080937D01FF9153
:10835000EF91BF91AF919F918F917F916F915F91BD
:108360004F913F912F910F900FBE0F901F90189536
:108370001F920F920FB60F9211248F939F938091AB
:10838000BC029091BD0201969093BD028093BC0205
:1083900080917B01882359F080917B0181508093EB
:1083A0007B0180917B01882311F481E08DBB9F913B
:1083B0008F910F900FBE0F901F9018951F920F92E4
:1083C0000FB60F9211248F939F93EF93FF93809199
:1083D000C0009091C6008C7181F480918803E82FD1
:1083E000F0E0E95FFC4F90838F5F8F778093880385
:1083F000809189038F5F80938903FF91EF919F9113
:108400008F910F900FBE0F901F9018951F920F9293
:108410000FB60F9211242F938F939F93EF93FF9397
:10842000209104032223B9F090910303E92FF0E097
:10843000ED53FD4F80818093C6009F5F90930303AF
:10844000822F815080930403882329F48091C100F6
:108450008F7D8093C100FF91EF919F918F912F911C
:108460000F900FBE0F901F9018951F920F920FB68E
:108470000F9211248F9380910403882349F48091F3
:10848000C1008F7B8093C1001092060310920503F8
:108490008F910F900FBE0F901F901895CF93DF9381
:1084A000EC0163E37BE044E050E00E940063892B31
:1084B00011F481E017C0CE016FE27BE043E050E0B1
:1084C0000E940063892B11F482E00CC0CE0168E2A7
:1084D0007BE046E050E00E940063892B11F483E0CA
:1084E00001C080E0DF91CF910895CF93DF93019792
:1084F00019F0C0E0D0E005C083E59DE00E9434188B
:10850000EC0187E39DE00E9434189E01280F391F7B
:10851000C901DF91CF910895A0E0B0E0E2E9F2E473
:108520000C948B623B01E82FFF27E7FDF095EE0FDF
:10853000FF1FED53F84F4590549086EF9DE00E9449
:1085400034184C01C2010E943418EC0188ED9DE002
:108550000E9434185C01C2010E9434186C018AEB3D
:108560009DE00E9434187C01C2010E9434188C01E5
:1085700086EA9DE00E943418C80DD91DCA0DDB1D86
:10858000CC0DDD1DCE0DDF1DC00FD11FC80FD91FB3
:1085900081E068167104A9F486E99DE00E94341810
:1085A0007C01C2010E9434188C018BE79DE00E947F
:1085B00034189701200F311F2C0F3D1F280F391F32
:1085C00007C086E79DE00E9434189C012C0F3D1FD8
:1085D000C901CDB7DEB7E0E10C94A762EF92FF923C
:1085E0000F931F93182F86E390E00E9402168EEDE2
:1085F00091E00E9434187C01E12FFF27E7FDF09500
:10860000EE0FFF1FE35CF74F859194910E943418A1
:108610008C018CE09EE00E9434180E0D1F1D080F87
:10862000191FC8011F910F91FF90EF900895A0E0CE
:10863000B0E0EDE1F3E40C949162082F86E390E062
:108640000E9402168EED91E00E9434185C01C02F4A
:10865000DD27C7FDD095CC0FDD1FFE01E35CF74F92
:10866000859194910E9434188C0188E49EE00E94C8
:1086700034186C01FE01ED53F84F859194910E94DE
:1086800034187C018AE39EE00E9434180A0D1B1DF9
:108690000C0D1D1D0E0D1F1D080F191FC801CDB794
:1086A000DEB7EAE00C94AD62AF92BF92CF92DF9258
:1086B000EF92FF920F931F938C01F62EE72E89ED18
:1086C0009CE00E9434185C01C8010E9434188C019F
:1086D0008FEC9CE00E9434186C01EF2DFE2DDF0121
:1086E0000D900020E9F71197AE1BBF0B8F2D9E2D2B
:1086F000BD010E9467157C0184EC9CE00E94341847
:108700000A0D1B1D0C0D1D1D0E0D1F1D080F191F21
:10871000C8011F910F91FF90EF90DF90CF90BF9015
:10872000AF900895A4E0B0E0E8E9F3E40C94996216
:10873000BE016F5F7F4F0E94513CCE01029662E006
:1087400070E00E9467152496E2E00C94B562A8E000
:10875000B0E0EDEAF3E40C948D627C01FC018081D1
:108760009181BE016F5F7F4F0E946D3CCE010296EA
:1087700064E070E00E9467153C018FE20E943015B2
:10878000F70182810E9492438C018FE20E94301592
:10879000F70183810E9492434C0180E20E943015D0
:1087A000F70184810E9492435C018AE30E943015A4
:1087B000F70185810E9492436C018AE30E94301583
:1087C000F70186810E949243080D191D0B5F1F4F10
:1087D0000A0D1B1D0C0D1D1D080F191F060D171D61
:1087E000C8012896EEE00C94A962A8E0B0E0EBEF97
:1087F000F3E40C9489626C0180E39DE00E943418DC
:108800009E838D83F601808191810E9434188C01B2
:1088100082E19DE00E94341898878F83F60182815F
:1088200093810E9434181C0189E09DE00E94341855
:108830002C01F60184817E010894E11CF11CB70132
:108840000E94513CF70101900020E9F73197EE19A1
:10885000FF09BF010E9467153C018BEF9CE00E945D
:1088600034184C01F6018581B7010E94513CF70193
:1088700001900020E9F73197EE19FF09BF010E942E
:1088800067155C0181EF9CE00E9434187C01F601C1
:1088900086819781FC01DF010D900020E9F7119797
:1088A000AE1BBF0BBD010E9467152D813E81020FDB
:1088B000131FEF81F8850E0F1F1F020D131D040DEE
:1088C000151D060D171D080D191D0A0D1B1D0E0D7A
:1088D0001F1D080F191FC8012896E2E10C94A5621C
:1088E000A8E2B0E0E6E7F4E40C949562082F1127C3
:1088F00007FD1095000F111FF801E75DFB4F8591F3
:108900009491F801E45BFE4F4591549139E0E32ED8
:10891000F12CEC0EFD1EB7010E94BF1BF801EF5DAC
:10892000FB4F859194919A838983F801E750FC4F1E
:10893000859194919C838B8381E28D838FE18E83DB
:10894000F886EF82CE0101960E94F543A896E6E0F4
:108950000C94B162A8E1B0E0E0EBF4E40C94956211
:10896000E82EFF24E7FCF0948701000F111FF801A7
:10897000ED56FC4F8591949101C0A895F999FDCFD2
:108980000E949D639B01AC012F3F8FEF38078FEF53
:1089900048078FEF580759F4F701EE0FFF1FEE0F4E
:1089A000FF1FE356FC4F2591359145915491F801F5
:1089B000ED51FC4F859194919A838983F801E75793
:1089C000FC4F859194919C838B8382E18D838FE012
:1089D0008E83CA01B901AE01475F5F4F0E94BF3E5F
:1089E00098878F83CE0101960E94F5436896E6E052
:1089F0000C94B162A0E0B0E0E0E0F5E40C94916288
:108A00005C0180E00E9417436C0180E00E94AA4450
:108A1000EC0181E00E94AA447C0182E00E94AA4409
:108A20008C0183E00E94AA44CC0DDD1DCE0DDF1D1C
:108A3000C00FD11FC80FD91F81E0A816B10419F4C7
:108A40008DE093E002C085E493E00E943418C80FE3
:108A5000D91F81E090E00E9475426091E804709116
:108A6000E904C80FD91F88E1AE010E94B322CDB737
:108A7000DEB7EAE00C94AD62AAE9B0E0E2E4F5E426
:108A80000C9489629C01880F991FBC01F3E0660F6A
:108A9000771FFA95E1F7680F791F6E537B4F70933C
:108AA000E9046093E804F901E251F94FE081E13013
:108AB00009F070C6232B29F0EAEE8E2EE5E09E2EFB
:108AC00004C07AEE872E74E0972EC4016AE879E03C
:108AD0000E940E63FC01108263ECE62E67E0F62E26
:108AE00000E0F70165917491C40146E050E00E94F6
:108AF0000063892B09F455C00F5F22E030E0E20EDD
:108B0000F31E063071F786E390E00E9402168EEDA8
:108B100091E00E9434182C018EEA99E00E943418EA
:108B2000480E591E882499248EE999E00E94341831
:108B30005C01F401ED53F84F859194910E94341833
:108B40008C018AE999E00E9434186C01F401E35C1D
:108B5000F74F859194910E9434187C0181E999E046
:108B60000E9434180A0D1B1D0C0D1D1D0E0D1F1D1E
:108B7000080F191F400E511E42E050E0840E951E52
:108B80005CE08516910481F680E090E00E947542D9
:108B90006091E8047091E904480E591E88E1A20131
:108BA0000DC657E0452E512C480C591C002309F0E6
:108BB00043C0D40117968C91882319F480E090E08B
:108BC00038C000E010E06E010894C11CD11C46E0E2
:108BD000842E912C800E911EF401E757FC4F659175
:108BE0007491C2010E940E637C01009701F103960B
:108BF000B6010E945B3E813079F4F401ED56FC4FE2
:108C00008591949101C0A895F999FDCF49815A8128
:108C10006B817C810E94CB630894E108F108F70125
:108C2000108202501040FFEF083F1F0781F681E0DD
:108C300090E00E94FA44C4C5013009F081C0D2011D
:108C40008C91882319F48824992459C0DE011C963C
:108C5000EEE8F1E088E001900D928150E1F732E119
:108C6000832E912C8C0E9D1E00E010E02CE3C22E72
:108C7000D12CCC0EDD1E90E2B92E86E0282E312CB0
:108C8000200E311EF101E750FC4F65917491C20135
:108C90000E940E637C01009779F1F6012B2D119251
:108CA0002A95E9F7BC016D5F7F4FC6010E94696399
:108CB000D4018D919C91B6010E946963F101E75D39
:108CC000FB4F6591749101C0A895F999FDCFC6013C
:108CD00040E250E00E94A9630894E108F108F7011E
:108CE0001082025010402EEF3FEF820E931E3FEF96
:108CF000083F130709F0C1CFB1E08B2E912C81E022
:108D00000E9417436C0180E00E9470442C0181E0B6
:108D10000E9470447C0182E00E9470448C0183E0D8
:108D20000E9470444C0C5D1C4E0C5F1C400E511E8A
:108D3000480E591E41E08416910409F07FC07BC0A3
:108D4000023009F08FC0D2018C91882319F4882455
:108D5000992445C0C20167EC79E00E940E637C0152
:108D60000097D1F105960E94123D90939B07809346
:108D70009A078F5F9F4F31F410929B0710929A07CA
:108D800001C0A895F999FDCF60919A0770919B0752
:108D900084EC90E00E94D7630894E108F108F701A1
:108DA0001082C20164EC79E00E940E630097A1F08A
:108DB0000396BE016F5F7F4F0E945B3E813061F47E
:108DC00001C0A895F999FDCF49815A816B817C81B9
:108DD00080EC90E00E94CB63A1E08A2E912C82E08F
:108DE0000E9417436C0184E00E94AA442C018CEC81
:108DF00099E00E9434187C018E010C5E1F4F809117
:108E00009A0790919B07B8010E946D3CF801019070
:108E10000020E9F73197E01BF10BC801BF010E9468
:108E200067154C0C5D1C4E0C5F1C480E591EF1E082
:108E30008F16910419F48DE093E002C085E493E06D
:108E40000E9434187C01E40CF51C81E090E00E9443
:108E500075426091E8047091E904E80EF91E88E11A
:108E6000A701ACC4033009F04FC1C2010E944E42B9
:108E7000813019F4F8E0FF2E05C0823011F40E9411
:108E8000B74FFF2483E00E94EE428C0189E39AE011
:108E90000E9434186091E8047091E904080F191FCA
:108EA00088E1A8010E94B322882309F089C486E3DF
:108EB00090E00E9402166F2CAA24BB24ECE22E2E16
:108EC000312C2C0E3D1E2F2D285FC656DF4F2883D8
:108ED000CA59D040E62DF0E074E0EE0FFF1F7A95FE
:108EE000E1F7DE015C96E058F64F80E101900D92CB
:108EF0008150E1F7DBA04C8C5D8C3E8DCE57DF4F6F
:108F00003883C258D0404F8DCF57DF4F4883C15868
:108F1000D04058A1C058DF4F5883C058D04079A0E6
:108F2000CAA08CA09DA08EA19FA1C258DF4F99839B
:108F30008883CE57D04080E19BE00E9434188C019A
:108F40006394862D0E9492437C0186E09BE00E9400
:108F50003418E00EF11EE80EF91E8D2D815083307D
:108F6000D8F45E824D82CE57DF4F9881C258D040F0
:108F70009F83CF57DF4FA881C158D040A887C058E2
:108F8000DF4FB881C058D040B9877A86CB86CE01F2
:108F900005960E94A74304C08FEF9AE00E94341800
:108FA000E80EF91E85EF9AE00E9434182701480E5A
:108FB000591EE2E0DE1661F486EE9AE00E94341853
:108FC0007C0189ED9AE00E943418E80EF91E77C002
:108FD000F1E0DF1609F06EC021E982162EE7920655
:108FE00044F08CEC9AE00E9434187C01E40CF51CEF
:108FF0005AC097FC02C08BE201C08DE20E9430157E
:10900000C40197FE03C0909581959F4FB1010E94C6
:109010006D3CF10101900020E9F73197E219F30965
:10902000C101BF010E9467154C0187EC9AE00E94C4
:1090300034186C01C258DF4F48815981CE57D04057
:1090400057FD02C08BE201C08DE20E943015C2586C
:10905000DF4F88819981CE57D04097FF03C090950C
:1090600081959F4FB1010E946D3CF101019000205C
:10907000E9F7E219F3093397CE018E96BF010E94FA
:1090800067158C0183EC9AE00E94341862E0E62EAA
:10909000F12CE40CF51CE80CF91CEC0CFD1CE00EAA
:1090A000F11EE80EF91E80EB9AE00E943418E80EDB
:1090B000F91E07C080EA9AE00E9434187C01E40C93
:1090C000F51C85E99AE00E943418E80EF91EAE0CF2
:1090D000BF1CC656DF4F5881CA59D040651609F0EB
:1090E000F9CE6091E8047091E90488E1A5010E943D
:1090F000B322882309F064C386E390E00E9402163D
:1091000083E060E070E098C1043009F09DC1C201C5
:109110000E944E42813039F488E0C856DF4F888380
:10912000C859D0400DC0823019F40E94AC4F03C022
:10913000833009F4179AC856DF4F1882C859D040B7
:1091400084E00E94EE428C0188E39BE00E94341888
:109150006091E8047091E904080F191F88E1A801E3
:109160000E94B322882309F02BC386E390E00E947B
:109170000216C956DF4F1882C759D040EE961FAE6F
:109180001EAEEE9754E1252E312C2C0E3D1E8EEC9A
:109190009BE00E9434188C01C956DF4FE881C75903
:1091A000D040C856DF4F9881C859D040E90FF0E051
:1091B00044E0EE0FFF1F4A95E1F7CF018058954F2D
:1091C000DC011C962D913D914D915C911F97CD56E0
:1091D000DF4F288339834A835B83C359D0401A9673
:1091E000CC901A971B96BC91C756DF4FB883C959CC
:1091F000D040DF01A857B54FEC901196DC90DC0110
:1092000016966C91169715965C91DF01AC57B54F89
:109210007C91DC0113964C911397EE57F54FE0814A
:109220002D913C9111971796FC90FF2009F4CAC02C
:109230008F2D8150843028F48AEB9BE00E943418F3
:109240000BC03E832D83EF83488779875A876B87CE
:10925000CE0105960E94A743080F191F80EB9BE0E3
:109260000E9434182C01EF2DF0E0EE0FFF1FEC5B95
:10927000F84F859194910E943418400E511E480E6B
:10928000591EB5E0FB1609F03FC08AEA9BE00E9438
:1092900034183C018E2D9D2DB1010E94D93BF10166
:1092A00001900020E9F73197E219F309C101BF01EC
:1092B0000E9467154C0184EA9BE00E9434185C010F
:1092C0008C2DC756DF4F9881C959D040B1010E94FB
:1092D000D93BF10101900020E9F73197E219F30938
:1092E000C101BF010E9467156C018DE99BE00E94DE
:1092F00034187C01CD56DF4F88819981C359D04005
:10930000B1010E94D93B41C0EAE0FE1621F0F7E02E
:10931000FF1609F05EC086E99BE00E9434183C010C
:109320008E2DB1010E94C13BF10101900020E9F7AF
:109330003197E219F309C101BF010E9467154C0181
:109340008FE89BE00E9434185C018C2DB1010E94D3
:10935000C13BF10101900020E9F73197E219F309CF
:10936000C101BF010E9467156C0187E89BE00E9464
:1093700034187C01CD56DF4F688179818A819B81C9
:10938000C359D040A1010E94033CF101019000208B
:10939000E9F73197E219F309C101BF010E9467158E
:1093A0008C0189E20E9430150894411C511C460C26
:1093B000571C480C591C4A0C5B1C4C0C5D1C4E0C79
:1093C0005F1C05C081E79BE00E9434182C01400E11
:1093D000511E86E69BE00E943418480E591EEE96F8
:1093E0002EAD3FADEE97240D351DEE963FAF2EAF5F
:1093F000EE97C956DF4F3881C759D0403F5FC956F5
:10940000DF4F3883C759D040383009F0C0CE609163
:10941000E8047091E90488E1EE964EAD5FADEE97F9
:109420000E94B322882309F0CBC186E390E00E941A
:10943000021684E061E070E00E948C428C0181E0C1
:1094400090E00E94754298C1053009F09EC185E008
:109450000E94EE42CF56DF4F99838883C159D04096
:1094600086E99CE00E9434188C016091AD047091F3
:10947000AE048091AF049091B0042CE3E22EF12C65
:10948000EC0EFD1EA7010E94BF3EBC018BE89CE0D4
:109490000E945443CD57DF4F99838883C358D040EF
:1094A0006091B1047091B2048091B3049091B404BE
:1094B000A7010E94BF3EBC018FE79CE00E9454437D
:1094C000CB57DF4F99838883C558D0406091B5044E
:1094D0007091B6048091B7049091B804A7010E94DE
:1094E000BF3EBC018FE69CE00E945443C957DF4F4A
:1094F00099838883C758D04060916109709162094F
:109500008091630990916409A7010E94BF3EBC014C
:1095100084E69CE00E945443C757DF4F99838883B9
:10952000C958D04087E59CE061E579E00E9454434A
:10953000C557DF4F99838883CB58D0408091670906
:10954000E82FF0E0E770F070EE0FFF1FEB55F74FDC
:1095500065917491C7010E94F06288E49CE0B701B4
:109560000E945443C357DF4F99838883CD58D0401E
:1095700080917D01E82FF0E0EE0FFF1FEA58F64FD3
:1095800065917491C7010E94F0628CE39CE0B70181
:109590000E945443C157DF4F99838883CF58D040EE
:1095A00080910001B7010E94C13B80910101BE0181
:1095B000625C7F4F0E94C13BB7016C5F7F4F80911F
:1095C00002010E94C13B8DE2FE01EE5BFF4F8083F2
:1095D000B701695F7F4F809103010E94C13BB701D2
:1095E000675F7F4F809104010E94C13BB701655FB7
:1095F0007F4F809105010E94C13BFE01E75BFF4F59
:10960000108280E39CE0B7010E9454431C0120912A
:109610001B04822F6AE00E942C62805D8CAF822F37
:109620000E942C62905D9DAF1EAE8EE19CE0B70162
:109630000E9454432C01C7016CE770E00E94F06265
:109640008DE09CE0B7010E9454433C01809070097A
:1096500090907109A0907209B0907309C501B4018E
:109660002CE330E040E050E00E946E62CA01B90194
:10967000A7010E94EC3C7CE5C72ED12CCC0EDD1E50
:10968000B7016B5F7F4FC6010E946963C60167E047
:109690007CE00E94DC62C501B4012CE330E040E0D4
:1096A00050E00E946E62DC01CB01B7010E946D3C6C
:1096B000C601BE01615C7F4F0E944A63C60162E041
:1096C0007CE00E94DC6283EF9BE0B6010E94544381
:1096D0006C0186EE9BE00E9434187C0181E090E0F2
:1096E0000E947542CF56DF4F48815981C159D04001
:1096F000040F151FCD57DF4FA881B981C358D04043
:109700000A0F1B1FCB57DF4FE881F981C558D040A6
:109710000E0F1F1FC957DF4F28813981C758D0400E
:10972000020F131FC757DF4F48815981C958D040D6
:10973000040F151FC557DF4FA881B981CB58D04002
:109740000A0F1B1FC357DF4FE881F981CD58D04066
:109750000E0F1F1FC157DF4F28813981CF58D040CE
:10976000020F131F020D131D040D151D060D171DED
:109770000C0D1D1D0E0D1F1D6091E8047091E90474
:10978000080F191F88E1A80119C06091E8047091C1
:10979000E90411C0E23079F486E390E00E940216F9
:1097A0008DE691E00E943418AC016091E80470915C
:1097B000E90488E103C081E140E050E00E94B32267
:1097C000C656DF4FE2E10C94A562682F88E046E7B9
:1097D00053E10E94211A0895E82FF0E0EE0FFF1FD9
:1097E000E65CFF4E4591549180E061E00E94211AB1
:1097F0000895E82FF0E0EE0FFF1FE357F04F45917B
:10980000549180E060E00E94211A0895A0E1B0E048
:10981000ECE0FCE40C949362E0907009F090710924
:109820000091720910917309C801B7012CE330E06F
:1098300040E050E00E946E62CA01B9016E010894D6
:10984000C11CD11CA6010E94EC3C80E061E0AE018D
:109850004A5F5F4F0E94311AC801B7012CE330E024
:1098600040E050E00E946E62DC01CB01B6010E9434
:109870006D3C8AE061E0AE014C5F5F4F0E94311A9F
:109880006096E8E00C94AF62A4E0B0E0EAE4FCE4A7
:109890000C949162B82EA62E6A01FA0180817E0195
:1098A0000894E11CF11CB7010E94513C8E010E5F2F
:1098B0001F4F8B2D6A2DA8010E94311A8AE30E9446
:1098C000C819F6018181B7010E94513CC8010E946C
:1098D000CF198AE30E94C819F6018281B7010E945C
:1098E000513CC8010E94CF192496EAE00C94AD6265
:1098F000A3E0B0E0EEE7FCE40C949462D82E7A0189
:109900008B0140348EE7580785E0680780E07807D0
:1099100038F088E06D2D4DE653E10E94211A2EC0EB
:10992000CB01BA0120E13EE040E050E00E946E62CF
:109930002983C801B70120E13EE040E050E00E94E9
:109940006E62162F072FF82EE92E2CE330E040E050
:1099500050E00E946E622A83612F702F8F2D9E2D02
:109960002CE330E040E050E00E946E626B8388E0C0
:109970006D2DAE014F5F5F4F0E94444C2396E7E090
:109980000C94B0628091D807813049F44091D1079E
:109990005091D2076091D3077091D4071BC08731D3
:1099A000E1F48091CD079091CE07A091CF07B091BF
:1099B000D0078F5F9F4FAF4FBF4F19F4EAE7F0E139
:1099C00015C04091C5075091C6076091C7077091B7
:1099D000C80781E00E94784C0895883119F4E8E7BF
:1099E000F0E104C0893139F4E6E7F0E145915491A2
:1099F00088E061E004C088E061E046E753E10E944E
:109A0000211A0895A3E2B0E0E8E0FDE40C9490622E
:109A1000082F0E94F019093018F4402F4F5C02C043
:109A2000402F49508FE060E00E943C1AE02FF0E0A8
:109A300044E0EE0FFF1F4A95E1F7DE011496E0586F
:109A4000F54F80E101900D928150E1F7DB849E811A
:109A5000CF809884A984BA848D2D8150843068F198
:109A60008D2D8550823248F534E1E32EF12CEC0E39
:109A7000FD1E892FB7010E94513C8E010B5E1F4FC6
:109A800080E060E0A8010E94311A8FE20E94C819AC
:109A90008C2DB7010E94513CC8010E94CF1980E271
:109AA0000E94C8199982AA82BB8286E060E0AE015A
:109AB0004F5F5F4F0E94444C06C080E060E042E58B
:109AC00053E10E94211AED2DF0E0EE0FFF1FEC5F35
:109AD000FC4E4591549180E061E00E94211AA396CA
:109AE000EBE00C94AC62A3E2B0E0E9E7FDE40C9497
:109AF0008F62182F0E94F0198BE00E94F94BE12F22
:109B0000F0E064E0EE0FFF1F6A95E1F7DE011496C6
:109B1000E058F64F80E101900D928150E1F7DB842F
:109B2000CE80BF8088849984AA8454E1E52EF12CEC
:109B3000EC0EFD1E812F8F5FB7010E94513C8E01FC
:109B40000B5E1F4F8EE060E0A8010E94311A80E09A
:109B500061E00E94F8198D2D8150823068F58C2DBE
:109B6000B7010E94513CC8010E94CF198FE20E94A8
:109B7000C8198B2DB7010E94513CC8010E94CF1912
:109B800080E20E94C81989829A82AB8286E061E0F5
:109B9000AE014F5F5F4F0E94444C80E20E94C819A3
:109BA00082E0D81611F482E404C081E0D81651F4A2
:109BB00082E50E94C81906C080E061E042E553E1F9
:109BC0000E94211AA396ECE00C94AB62A3E1B0E0F2
:109BD000ECEEFDE40C948D6280917509E82FF0E0C5
:109BE000EE0FFF1FEC56FF4E65917491CE01089663
:109BF0000E94F06260901D0170901F018090210111
:109C0000A0902901B0902A01009125011091260110
:109C10000F5F1F4F909023018091270190912801A1
:109C2000FCE0CF2ED12CCC0EDD1E8459984FB6010E
:109C30000E946D3CEDE0EE2EF12CEC0EFD1E80E05E
:109C400060E0A7010E94311A8FE20E94C819802F9C
:109C5000B6010E94513CC7010E94CF198FE20E94B9
:109C6000C819892DB6010E94513CC7010E94CF1925
:109C700080E20E94C8198E010C5F1F4FAA0CBB1C0A
:109C8000AA0CBB1C8FE59EE0A80EB91EC801B50149
:109C90000E94F062C8010E94CF1980E20E94C81998
:109CA00000916709077091F480910601803C11F4DE
:109CB00081E415C0803411F489E411C0803811F4B6
:109CC00084E40DC080917407805D09C0013011F4F7
:109CD00082E505C0023011F08AE401C087E40E94E9
:109CE000C81989827A826B8280E061E0AE014F5FA1
:109CF0005F4F0E94444C80E20E94C819CE01089632
:109D00000E94CF1980E20E94C819023060F480914D
:109D10000701BE016C5F7F4F0E94513CCE0105964A
:109D20000E94CF1921C00230C9F48091670988735D
:109D300021F486E40E94C8190FC0883011F482E52E
:109D400003C0803189F48AE50E94C81980916709AF
:109D500086FF02C082E506C086E404C080E30E945C
:109D6000C81981E30E94C819E0917D01F0E0E5582F
:109D7000F14FE4918E2F0E94C8196396EEE00C9487
:109D8000A962A0E1B0E0E7ECFEE40C9493620091DC
:109D900065090E94F019002319F40E94E64DD8C00D
:109DA000013019F580E060E041E40E943C1A6091C6
:109DB000AD047091AE048091AF049091B0048E0117
:109DC0000F5F1F4FA8010E94BF3E0E94CF1980E085
:109DD00061E04DE40E943C1A6091B1047091B204BC
:109DE0008091B3049091B40424C0023041F580E026
:109DF00060E047E40E943C1A6091B5047091B6049B
:109E00008091B7049091B8048E010F5F1F4FA80195
:109E10000E94BF3E0E94CF1980E061E044E40E94AE
:109E20003C1A609161097091620980916309909177
:109E30006409A8010E94BF3E0E94CF1989C0033067
:109E400079F581E00E94F94B80911B046AE00E9441
:109E50002C62805D0E94C81980911B046AE00E94F8
:109E60002C62892F805D0E94C81983E00E94EC4B10
:109E700004E0B0E0EB2EB1E0FB2E6E010894C11CB3
:109E8000D11CF70181917F01B6010E94C13BAC0159
:109E9000802F61E00E94311A0E5F003191F758C0A7
:109EA000043061F480E060E041E559E00E94311A3D
:109EB00084E00E94EC4B0E94C24C4AC0053091F5F0
:109EC00086E00E94F94B809167098770823031F0FB
:109ED000813021F080917609882391F188E060E05B
:109EE00046E753E10E94211A85E00E94EC4B8091E5
:109EF0009A0790919B07892B71F080917709909137
:109F00007809019741F40E948C0EAB01BC0181E0FD
:109F10000E94784C1DC088E061E046E753E10E9452
:109F2000211A16C00630A1F48CE00E94F94B85E09E
:109F300061E041E653E10E94211A0E94064C08C0EC
:109F40000E94A70EAB01BC0180E00E94784CCCCFF0
:109F50006096E8E00C94AF6280E091E0E0E8FAE01F
:109F6000DF019C011D9221503040E1F7089580E00F
:109F700091E0E0E8F9E0DF019C011D9221503040C2
:109F8000E1F70895EF92FF920F931F93182F80E946
:109F90009AE060E87AE040EF50E00E94316360911F
:109FA000270170912801E0912501E0902301F090B4
:109FB000210100911F01F0911D01153079F44091AC
:109FC00015045091160420911304309114048091CB
:109FD000110490911204A0E0B0E032C01A3011F0E8
:109FE000173089F48091BC04482F50E08091BD0463
:109FF000282F30E08091BE049091BF04A091C0044E
:10A00000B091C1041DC0812F8850823048F080E09B
:10A0100090E0A0E0B0E020E030E040E050E010C090
:10A0200040912E0450912F0420912C0430912D0446
:10A030008091240490912504A0912604B0912704D6
:10A0400080938C0A90938D0AA0938E0AB0938F0A06
:10A0500030938B0A20938A0A5093890A4093880A86
:10A060001093870AF093860A0093850AF092840A77
:10A07000E092830AEF5FE093820A6459784F70930D
:10A08000810A6093800A1A3079F01B3169F011322D
:10A0900059F01C3049F01D3039F0113029F01230E0
:10A0A00019F0143009F017981F910F91FF90EF905D
:10A0B0000895FF920F931F93F82E80E999E08C0189
:10A0C00000511040B80140EF50E00E943163809190
:10A0D0002701909128018459984F509125015F5F85
:10A0E000B0912301A0912101F0911F01E0911D0188
:10A0F0006091760770917707209178073091790702
:10A100004091750710928F0910928E0910928D0957
:10A1100040938C09F092870930938B0920938A0928
:10A120007093890960938809E0938609F093850903
:10A13000A0938409B093830950938209F801918315
:10A1400080831F910F91FF9008951F93CF93DF930A
:10A15000EC01162F1092940B1E860C960E94123D55
:10A160008E3391050CF066C0909366018093650173
:10A170001C86CE010A960E94123D8C3391050CF08C
:10A1800059C090936801809367011A86CE010896A2
:10A190000E94123D883191050CF04CC090936A01E9
:10A1A000809369011886CE0106960E94123D0097A1
:10A1B00009F440C080329105ECF590936C018093D6
:10A1C0006B011E82CE0104960E94123D01978C30D5
:10A1D000910584F590936E0180936D011C82CE01F0
:10A1E0000E94123D8C5697409093700180936F01AE
:10A1F0001092720110927101109274011092730109
:10A2000085E691E00E94B11D60938E0B70938F0BD9
:10A210008093900B9093910B80918E0B90918F0B6C
:10A22000A091900BB091910BB7FD02C01093940BCD
:10A2300081E001C080E0DF91CF911F910895AF923E
:10A24000BF92CF92DF92EF92FF920F931F93379BB3
:10A2500008C010927A091092790989E080937D01F3
:10A260007AC180917D01893019F482E080937D016B
:10A2700010917609112309F46EC11130D9F41092AE
:10A28000940B0E94031B8091790990917A09892B84
:10A2900019F483EA93E102C08CE993E10E942C1C3B
:10A2A00082E0809376090E94C91A90937C0980937A
:10A2B0007B0951C11230D9F50E94171B813009F07A
:10A2C00034C18091790990917A09892BC1F48AE887
:10A2D00093E066E973E145E050E00E940063892B5A
:10A2E00039F481E090E090937A098093790911C064
:10A2F00080E490E00E94C40E10937D0113C18AE8AF
:10A3000093E06DE873E148E050E00E940063892B20
:10A3100011F483E052C0A1E4B1E0EDE1F1E082E1AB
:10A3200001900D928150E1F71092760915C113301A
:10A3300041F40E94031B86E893E10E942C1C84E0F8
:10A34000B0CF143009F051C00E94171B813009F0C2
:10A350003FC01092940382E993E00E94123D00975F
:10A3600079F18032910564F590936C0180936B01D3
:10A37000109291038FE893E00E94123D01978C3078
:10A380009105F4F490936E0180936D0110928E0309
:10A390008AE893E00E94123D8C56974097FD10C0CA
:10A3A0009093700180936F0110927201109271016D
:10A3B000109274011092730185E080937609CBC0EE
:10A3C00080E490E00E94C40E81E080937D01AAC0E9
:10A3D0000E94C91A20917B0930917C09821B930B42
:10A3E000805D974008F4B7C0ABC0153041F40E94BF
:10A3F000031B8FE793E10E942C1C86E052CF16309E
:10A4000009F0A9C00E94171B813009F08EC010927C
:10A41000920380E993E00E94123D8C3391050CF089
:10A4200081C0909366018093650110928F038DE83F
:10A4300093E00E94123D8C3391050CF073C0909311
:10A4400068018093670110928C038AE893E00E9470
:10A45000123D883191050CF065C090936A0180939C
:10A46000690185E691E00E94B11D7B018C0180E7C6
:10A47000A82E81E8B82E8FEFC82E8FEFD82EEA0CC9
:10A48000FB1C0C1D1D1D17FD48C0F8942091820B6C
:10A490003091830B4091840B5091850B789480917F
:10A4A0001B0190911C01892B01F580919F079091D0
:10A4B000A0070097D1F057016801A21AB30AC40A95
:10A4C000D50AA6019501D7FE07C050954095309555
:10A4D00021953F4F4F4F5F4FA0E0B0E082179307A9
:10A4E000A407B50714F482E019C0E0928E0BF09235
:10A4F0008F0B0093900B1093910B81E08093940B42
:10A5000010927907109278071092770710927607C9
:10A5100010927D0110927C0105C081E080937D0145
:10A520000E949D0B1092760916C00E94C91A2091B4
:10A530007B0930917C09821B930B805D974058F01A
:10A5400080E490E00E94C40E83E080937D0110922D
:10A55000760985E201C080E01F910F91FF90EF9096
:10A56000DF90CF90BF90AF900895A1E0B0E0EBEB0B
:10A57000F2E50C948F62182F0E94031B183019F417
:10A580008FE094E106C0103111F0CC244BC08BED6C
:10A5900093E10E942C1C0E94C91A5C018C01CC24FE
:10A5A000DD244E010894811C911C02C0DD2487012A
:10A5B0000E94C91A7C010817190709F0A895C7015C
:10A5C0008A199B09805D974018F025E2C22E2AC0A7
:10A5D000DD2059F4C4010E94E61A813041F78981D7
:10A5E000843229F7DD24D394E2CF81E0D81669F4D0
:10A5F0000E94171BC82E21E0821719F492E0D92E71
:10A60000D6CF82E0C81699F60DC022E0D21679F6B0
:10A610008AE893E06DEC73E14DE050E00E94006346
:10A62000892B21F68C2D2196ECE00C94AB62A0E1F5
:10A63000B0E0EDE1F3E50C9496628AE893E06CE219
:10A6400070E00E945563009709F49DC08C010F5F74
:10A650001F4FCE010996B80146E050E00E947E638C
:10A66000C8016CE270E00E945563FC01009709F498
:10A670008AC0F18001966CE270E00E9455630097F9
:10A6800009F481C001966CE270E00E945563009766
:10A6900009F479C001966CE270E00E94556300975E
:10A6A00009F471C001966CE270E00E945563009756
:10A6B00009F469C001966CE270E00E94556300974E
:10A6C00009F461C001966CE270E00E945563009746
:10A6D00009F459C001966CE270E00E9455638C0148
:10A6E000009709F450C0BC016F5F7F4FCE01079601
:10A6F00042E050E00E947E63B8016D5F7F4FCE0163
:10A70000059642E050E00E947E63B8016B5F7F4F88
:10A71000CE01039642E050E00E947E63F8018581FD
:10A72000873324F081E3898389E303C082E389834B
:10A7300080E38A83CE01019661E070E00E94A5501B
:10A74000882311F482E220C0F1E4FF1661F48091C5
:10A75000930B882311F087E001C086E080937D0190
:10A7600010927C010EC086E5F81669F488E08093AB
:10A770007D0180916A0990916B09892B89F30E9470
:10A780009D0B80E001C083E26096E5E00C94B2622C
:10A79000A0E1B0E0EEECF3E50C94956288E08093E4
:10A7A0007D018AE893E06CE270E00E9455630097B7
:10A7B00091F08C010F5F1F4FCE010996B80146E062
:10A7C00050E00E947E63C8016CE270E00E94556315
:10A7D0007C01009721F40E949D0B83E239C008940C
:10A7E000E11CF11CCE010796B70142E050E00E9447
:10A7F0007E6383E090E0E80EF91ECE010596B70176
:10A8000042E050E00E947E6383E090E0E80EF91E93
:10A810008E010F5F1F4FC801B70144E050E00E9456
:10A820007E63C80161E070E00E94A550882321F496
:10A830000E949D0B82E20CC08091930B882311F043
:10A8400087E001C086E080937D0110927C0180E06A
:10A850006096E6E00C94B162FC01808191819A32AD
:10A8600039F09A3029F03196992311F08927F6CFE3
:10A870000E94C13B0895A5E0B0E0E1E4F4E50C944A
:10A88000986280910D0490910E04892BD1F4CE0131
:10A8900001960E94E61A813009F0F1C08981843264
:10A8A00009F0EDC00E94C91A90930C0480930B0428
:10A8B00081E090E090930E0480930D0410920A04BE
:10A8C000DEC00E94171B813009F0C8C010916709D3
:10A8D000187309F069C08AE893E062EC73E14AE01A
:10A8E00050E00E940063892B09F0C9C09091950344
:10A8F000993331F481E3809393039093940306C0DA
:10A9000082E38093930380E38093940383E993E04D
:10A9100062E070E00E94A550813011F082E2B2C086
:10A92000F8941092810B1092800B80918E0B909175
:10A930008F0BA091900BB091910B80938E07909309
:10A940008F07A0939007B09391078093820B909309
:10A95000830BA093840BB093850B78948091A20312
:10A96000813311F484E00EC0823321F485E08093BA
:10A970007D0117C0833309F082C08091A403803326
:10A9800051F486E080937D0180916A0990916B0972
:10A99000892B39F403C087E080937D0110927C01FC
:10A9A0006EC00E949D0B6BC08AE893E0BE016E5F93
:10A9B0007F4F0E942C548AE893E06AE270E00E9484
:10A9C0005563FC0191818A81981709F05AC09281E0
:10A9D0008B81981709F055C08AE893E066E971E029
:10A9E00044E050E00E947063009731F48091670961
:10A9F00080688093670943C01830B9F48AE893E00F
:10AA00006CEB73E145E050E00E940063892B51F04C
:10AA10008AE893E066EB73E145E050E00E94006352
:10AA2000892B69F50E9417532DC0103141F58AE832
:10AA300093E060EB73E145E050E00E940063892BF6
:10AA400051F08AE893E06AEA73E145E050E00E9441
:10AA50000063892BA1F40E94C85314C00E94C91A34
:10AA600020910B0430910C04821B930B885E934061
:10AA700030F010920E0410920D0485E203C080E0C5
:10AA800001C084E22596E3E00C94B462A8E0B0E053
:10AA9000ECE4F5E50C94956281E00E941B1A81E0DC
:10AAA00061E041EC56E10E94211A80916A0990917F
:10AAB0006B097E010894E11CF11CB7010E946D3CFA
:10AAC000AC0186E061E00E94311A86E061E0A701F6
:10AAD00025E000E010E00E948C3F892B19F421E072
:10AAE00030E012C0C7010E94123DBC0190936B0977
:10AAF00080936A0901C0A895F999FDCF82ED90E095
:10AB00000E94D76320E030E0C9012896E6E00C946B
:10AB1000B162A8E0B0E0EFE8F5E50C94956281E061
:10AB20000E941B1A81E061E04FEC56E10E94211A5D
:10AB300080916809909169097E010894E11CF11CDB
:10AB4000B7010E946D3CAC0186E061E00E94311AC1
:10AB500086E061E0A70125E000E010E00E948C3F64
:10AB6000892B19F421E030E012C0C7010E94123D88
:10AB7000BC01909369098093680901C0A895F9996F
:10AB8000FDCF80ED90E00E94D76320E030E0C90166
:10AB90002896E6E00C94B1621F93182F0E94F019DA
:10ABA000E12FF0E0EE0FFF1FEE5BFA4E459154915E
:10ABB00080E060E00E94211A1F910895EF92FF92B9
:10ABC0001F93DF93CF930F92CDB7DEB78FE00E9434
:10ABD000CC5510910F04E12FF0E0EE0FFF1FEC5663
:10ABE000F94E4591549180E061E00E94211A7E0166
:10ABF0000894E11CF11C812F67E0A7010E94693FC6
:10AC0000182F8981893109F45CC0843109F049C069
:10AC100010930F04809167098770823079F5109244
:10AC2000C100112319F484E395E01DC0113019F41B
:10AC30008AE992E018C0123019F48CE491E013C054
:10AC4000133019F485EA90E00EC0143019F482E54F
:10AC500090E009C0153019F489E290E004C0163084
:10AC600031F48BE190E09093C5008093C40088E9B3
:10AC70008093C1008091C60001C0A895F999FDCFCD
:10AC800086E090E00E94A363792F01C0A895F9990E
:10AC9000FDCF86E090E0612F0E94D76320E030E096
:10ACA00012C081E00E941B1AE12FF0E0EE0FFF1F9F
:10ACB000EC56F94E4591549180E061E00E94211AD2
:10ACC0009ACF21E030E0C9010F90CF91DF911F9121
:10ACD000FF90EF900895A8E0B0E0E1E7F6E50C946E
:10ACE00095628EE00E94CC5581E061E042EA56E137
:10ACF0000E94211A80919F079091A0077E010894DD
:10AD0000E11CF11CB7010E946D3CAC0187E061E0E1
:10AD10000E94311A87E061E0A70125E000E010E021
:10AD20000E948C3F892B19F421E030E012C0C7014A
:10AD30000E94123DBC019093A00780939F0701C021
:10AD4000A895F999FDCF88EC90E00E94D76320E0A8
:10AD500030E0C9012896E6E00C94B162A8E0B0E0CA
:10AD6000E4EBF6E50C9495628DE00E94CC5581E011
:10AD700061E041EB56E10E94211A80919807909181
:10AD800099077E010894E11CF11CB7010E946D3CFB
:10AD9000AC0189E061E00E94311A89E061E0A7011D
:10ADA00025E000E010E00E948C3F892B19F421E09F
:10ADB00030E012C0C7010E94123DBC019093990778
:10ADC0008093980701C0A895F999FDCF86EC90E093
:10ADD0000E94D76320E030E0C9012896E6E00C9499
:10ADE000B162EF92FF921F93DF93CF930F92CDB793
:10ADF000DEB78CE00E94CC558091670990E056E068
:10AE0000969587955A95E1F7182F1170E12FF0E08C
:10AE1000EE0FFF1FEF5DF94E4591549180E061E028
:10AE20000E94211A7E010894E11CF11C812F62E02E
:10AE3000A7010E94693F182F89818931A1F18431CE
:10AE400011F501C0A895F999FDCF8CE390E00E941F
:10AE5000A36320916709112331F42F7B20936709A5
:10AE6000BC01677F07C0206420936709BC0168604C
:10AE700001C0A895F999FDCF8CE390E00E94D763BB
:10AE800020E030E012C081E00E941B1AE12FF0E0C8
:10AE9000EE0FFF1FEF5DF94E4591549180E061E0A8
:10AEA0000E94211AC3CF21E030E0C9010F90CF9159
:10AEB000DF911F91FF90EF900895EF92FF921F9303
:10AEC000DF93CF930F92CDB7DEB78BE00E94CC55C6
:10AED000109167091695169516951770E12FF0E0F9
:10AEE000EE0FFF1FE95FF94E4591549180E061E05C
:10AEF0000E94211A7E010894E11CF11C812F63E05D
:10AF0000A7010E94693F182F8981893109F43AC04D
:10AF1000843141F501C0A895F999FDCF8CE390E00B
:10AF20000E94A363BC01687F80916709877C11231D
:10AF300019F4809367090DC0113029F4886080935B
:10AF40006709616006C0806180936709626001C023
:10AF5000A895F999FDCF8CE390E00E94D76320E09B
:10AF600030E012C081E00E941B1AE12FF0E0EE0FEA
:10AF7000FF1FE95FF94E4591549180E061E00E9426
:10AF8000211ABCCF21E030E0C9010F90CF91DF91B1
:10AF90001F91FF90EF900895CF92DF92FF920F9351
:10AFA0001F93DF93CF930F92CDB7DEB788E00E9457
:10AFB000CC55F0907509EF2DF0E0EE0FFF1FE8542F
:10AFC000FA4E4591549180E061E00E94211A6E0191
:10AFD0000894C11CD11C8F2D66E0A6010E94693F18
:10AFE000F82E8981893109F434C00F2D10E08431A5
:10AFF00009F5F0927509F801EE0FFF1FEE0FFF1F24
:10B00000EC53FA4E85919591A591B4918093770177
:10B0100090937801A0937901B0937A0101C0A8952B
:10B02000F999FDCF8CEC90E0B8010E94D76320E045
:10B0300030E011C081E00E941B1AF801EE0FFF1FE3
:10B04000E854FA4E4591549180E061E00E94211A43
:10B05000C2CF21E030E0C9010F90CF91DF911F9165
:10B060000F91FF90DF90CF900895CF92DF92FF92E3
:10B070000F931F93DF93CF930F92CDB7DEB787E087
:10B080000E94CC5501C0A895F999FDCF8AEC90E0BB
:10B090000E94A3638C01FF24F394F822EF2DF0E0CB
:10B0A000EE0FFF1FEF5AF94E4591549180E061E099
:10B0B0000E94211A6E010894C11CD11C8F2D62E0E0
:10B0C000A6010E94693FF82E8981893191F184316E
:10B0D00001F580916709982F9770FF2031F4B8012E
:10B0E0006E7F913061F4887F06C0B801616099235A
:10B0F00031F4887F81608093670901C0A895F99930
:10B10000FDCF7F778AEC90E00E94D76320E030E0AB
:10B1100012C081E00E941B1AEF2DF0E0EE0FFF1F1E
:10B12000EF5AF94E4591549180E061E00E94211A56
:10B13000C5CF21E030E0C9010F90CF91DF911F9181
:10B140000F91FF90DF90CF900895A8E0B0E0EBEA78
:10B15000F8E50C94956286E00E94CC5580E061E0B1
:10B160004DED56E10E94211A80919A0790919B071C
:10B170007E010894E11CF11CB7010E946D3CAC01FA
:10B1800089E061E00E94311A89E061E0A70125E0D1
:10B1900000E010E00E948C3F892B19F421E030E0A0
:10B1A00012C0C7010E94123DBC0190939B0780937F
:10B1B0009A0701C0A895F999FDCF84EC90E00E9410
:10B1C000D76320E030E0C9012896E6E00C94B16234
:10B1D000A4E1B0E0EEEEF8E50C9493626B010E94FE
:10B1E000CC5501C0A895F999FDCFC6010E949D6379
:10B1F00069837A838B839C8325E0E22EF12CEC0E0D
:10B20000FD1EA7010E94BF3E81E061E0A7012FE083
:10B2100000E010E00E948C3F892B19F421E030E01F
:10B2200015C0C701BE016F5F7F4F0E945B3E81303A
:10B2300059F401C0A895F999FDCF49815A816B81D4
:10B240007C81C6010E94CB6320E030E0C901649696
:10B25000E8E00C94AF6285E060EC70E00E94E85892
:10B26000089583E06CE270E00E94E858089582E05F
:10B2700068E270E00E94E858089581E064E270E0BE
:10B280000E94E858089580E060E270E00E94E8586B
:10B290000895CF92DF92FF920F931F93DF93CF9386
:10B2A0000F92CDB7DEB784E00E94CC5501C0A895BF
:10B2B000F999FDCF8CE090E00E94A3638C01F12E00
:10B2C000FF1CFF24FF1CEF2DF0E0EE0FFF1FEC5CD6
:10B2D000F94E4591549180E061E00E94211A6E017F
:10B2E0000894C11CD11C8F2D62E0A6010E94693F09
:10B2F000F82E8981893141F18431B1F4FF2029F49C
:10B300001092D807B8017F7706C08093D807B8019C
:10B31000706801C0A895F999FDCF8CE090E00E947B
:10B32000D76320E030E012C081E00E941B1AEF2DAD
:10B33000F0E0EE0FFF1FEC5CF94E4591549180E078
:10B3400061E00E94211ACFCF21E030E0C9010F90C7
:10B35000CF91DF911F910F91FF90DF90CF900895D3
:10B36000A4E0B0E0E6EBF9E50C949862182F0E9497
:10B37000F01980E060E041EF56E10E94211AE12FD0
:10B38000FF27E7FDF095EE0FFF1FEE5BFA4E4591AC
:10B39000549180E061E00E94211A812F8F5FBE01ED
:10B3A0006F5F7F4F0E94513C8BE060E0AE014E5FCB
:10B3B0005F4F0E94311A8DE060E04DEE56E10E9431
:10B3C000211A2496E3E00C94B462CF92DF92FF92AC
:10B3D0000F931F93DF93CF93CDB7DEB7A1970FB62F
:10B3E000F894DEBF0FBECDBFDE011296EBE9F1E0AF
:10B3F00080E201900D928150E1F70E94B059FF2444
:10B400006E010894C11CD11C8F2D61E1A6010E9420
:10B41000693FF82E89818931C1F0843119F000E04B
:10B4200010E00EC080E1F81681F0EF2DF0E0EE0F95
:10B43000FF1FEC0DFD1D0180F281E02D09958C01AF
:10B440008F2D0E94B059012BF9F28091D8078823E3
:10B4500009F045C01092DA071092D90780E290E017
:10B4600044E651E068EA70EC0E94051C6093AD046C
:10B470007093AE048093AF049093B00484E290E0A4
:10B4800040E05FEF6FEF7FEF0E94051C6093B10417
:10B490007093B2048093B3049093B40488E290E074
:10B4A00041E051E068EA70EC0E94051C6093B5042D
:10B4B0007093B6048093B7049093B8048CE290E044
:10B4C00041E051E068EA70EC0E94051C609361095C
:10B4D00070936209809363099093640917C0843163
:10B4E000A9F481E090E09093DA078093D907A8E06F
:10B4F000B1E0EDE1F1E082E101900D928150E1F7E0
:10B500000E942A28882311F00E94C24FA1960FB6EC
:10B51000F894DEBF0FBECDBFCF91DF911F910F9189
:10B52000FF90DF90CF900895EF92FF920F93DF93FB
:10B53000CF93CDB7DEB760970FB6F894DEBF0FBEDE
:10B54000CDBFA82F002309F461C07E010894E11C3F
:10B55000F11C88E0F70111928A95E9F729833A8373
:10B560004B835C836D837E83AF83988780E2801BEF
:10B57000E82FFF27E7FDF09549815A816B817C8197
:10B58000181684F019861A861B861C868827992728
:10B590008E1B9F0B04C0440F551F661F771F8A9593
:10B5A000D2F728C0202F332727FD3095DB01CA01B1
:10B5B000022E04C0880F991FAA1FBB1F0A94D2F73E
:10B5C00089879A87AB87BC8704C07695679557951E
:10B5D0004795EA95D2F78D819E81AF81B88504C0E9
:10B5E000880F991FAA1FBB1F2A95D2F7482B592BEA
:10B5F0006A2B7B2B4D875E876F87788B29853A85F1
:10B600004B855C856D857E85AF8598898A2F609690
:10B610000FB6F894DEBF0FBECDBFCF91DF910F9173
:10B62000FF90EF900895EF92FF920F93DF93CF93E7
:10B63000CDB7DEB760970FB6F894DEBF0FBECDBFB3
:10B64000A82F002309F467C07E010894E11CF11CB7
:10B6500088E0F70111928A95E9F729833A834B83B1
:10B660005C836D837E83AF83988780E2801B4D81EE
:10B670005E816F817885E82FFF27E7FDF09518162A
:10B68000B4F0DB01CA01BB0F880B982FDC018D875A
:10B690009E87AF87B88B882799278E1B9F0B04C086
:10B6A00075956795579547958A95D2F728C0202FAD
:10B6B000332727FD3095DB01CA01022E04C0B59562
:10B6C000A795979587950A94D2F78D879E87AF8720
:10B6D000B88B04C0440F551F661F771FEA95D2F739
:10B6E00089819A81AB81BC8104C0B695A795979555
:10B6F00087952A95D2F7482B592B6A2B7B2B4987A4
:10B700005A876B877C8729853A854B855C856D8553
:10B710007E85AF8598898A2F60960FB6F894DEBF34
:10B720000FBECDBFCF91DF910F91FF90EF900895A5
:10B73000AEE5B0E0EEE9FBE50C948962A8E04E01CD
:10B740000894811C911CF4016A2E11926A94E9F705
:10B7500029833A834B835C836D837E838F839887B1
:10B76000CE010996FC011192AA95E9F7A986BA863D
:10B77000CB86DC86ED86FE860F87188B29843A847B
:10B780004B845C84ED84FE840F85188969807A80FF
:10B790008B809C806DA67EA68FA698AA6D807E80E9
:10B7A0008F809884E114F1040105110509F0B3C3F9
:10B7B000621473048404950408F03DC100E020166F
:10B7C00000E0300601E0400600E0500688F41FEF7C
:10B7D000211631044104510439F030F048E0E42EE0
:10B7E000F12C012D112D18C0EE24FF24870114C067
:10B7F00020E0221620E0320620E0420621E0520638
:10B8000030F038E1E32EF12C012D112D05C020E19F
:10B81000E22EF12C012D112DD201C1010E2C04C0FC
:10B82000B695A795979587950A94D2F785549E4F1C
:10B83000DC012C9180E290E0A0E0B0E08E199F093D
:10B84000A00BB10B7C018D01E21AF108010911096D
:10B85000E114F10401051105A1F10E2C04C0220C24
:10B86000331C441C551C0A94D2F7A40193010E2CDE
:10B8700004C0220F331F441F551F0A94D2F780E2E1
:10B8800090E08E199F096DA47EA48FA498A804C08F
:10B8900096948794779467948A95D2F7622A732A4C
:10B8A000842A952AADA4BEA4CFA4D8A804C0AA0C0B
:10B8B000BB1CCC1CDD1CEA94D2F7ADA6BEA6CFA65D
:10B8C000D8AA6201EE24FF24CDAADEAAEFAAF8AE20
:10B8D000920181012070307009AF1AAF2BAF3CAFDD
:10B8E000C401B301A70196010E944C627B018C0147
:10B8F000C401B3012DA93EA94FA958AD0E944C62C5
:10B90000C901DA013C014D01C401B30129AD3AADD1
:10B910004BAD5CAD0E940D629B01AC018701FF2421
:10B92000EE24ADA4BEA4CFA4D8A8C601AA27BB27E5
:10B9300057016801A82AB92ACA2ADB2AA216B30627
:10B94000C406D506E0F408946108710881089108DE
:10B95000A20CB31CC41CD51CA214B304C404D5048B
:10B9600070F0A216B306C406D50648F40894610820
:10B97000710881089108A20CB31CC41CD51CA21A22
:10B98000B30AC40AD50AC601B5012DA93EA94FA91B
:10B9900058AD0E944C627B018C01C601B5012DA9F6
:10B9A0003EA94FA958AD0E944C62C901DA015C0161
:10B9B0006D01C601B50129AD3AAD4BAD5CAD0E943C
:10B9C0000D629B01AC018701FF24EE248DA59EA58D
:10B9D000AFA5B8A9A070B070E82AF92A0A2B1B2BD2
:10B9E000E216F30604071507C0F40894A108B1088D
:10B9F000C108D108E20CF31C041D151DE214F30468
:10BA00000405150550F0E216F3060407150728F49F
:10BA10000894A108B108C108D108D3019927882743
:10BA200086017501E82AF92A0A2B1B2BE9AAFAAA32
:10BA30000BAB1CABCFC4211431044104510471F48D
:10BA400061E070E080E090E020E030E040E050E035
:10BA50000E944C62C901DA011C012D0100E0201690
:10BA600000E0300601E0400600E0500688F41FEFD9
:10BA7000211631044104510431F028F048E050E02F
:10BA800060E070E017C040E050E060E070E012C09D
:10BA900020E0221620E0320620E0420621E0520695
:10BAA00028F048E150E060E070E004C040E150E080
:10BAB00060E070E0D201C101042E04C0B695A795E4
:10BAC000979587950A94D2F785549E4FDC012C9167
:10BAD000E0E2EE2EF12C012D112DD801C701841BBF
:10BAE000950BA60BB70B821B9109A109B109009711
:10BAF000A105B10561F464015301A218B308C4089B
:10BB0000D50831E0632E712C812C912C1EC16F96CB
:10BB10008FAF6F97082E04C0220C331C441C551C99
:10BB20000A94D2F7EE2DE81B640153010E2E04C0D7
:10BB3000D694C794B794A7940A94D2F7A40193011A
:10BB40006F960FAC6F9704C0220F331F441F551F11
:10BB50000A94D2F76DA47EA48FA498A80E2E04C0D8
:10BB600096948794779467940A94D2F7840173012A
:10BB7000E22AF32A042B152BE9A6FAA60BA71CA789
:10BB8000320188249924920181012070307021961D
:10BB90000CAF1DAF2EAF3FAF2197C601B501A40179
:10BBA00093010E944C627B018C01C601B501A40186
:10BBB00093010E944C62C901DA0125968CAF9DAFBA
:10BBC000AEAFBFAF2597BC01CD0121962CAD3DADE9
:10BBD0004EAD5FAD21970E940D629B01AC018701C4
:10BBE000FF24EE24A9A4BAA4CBA4DCA4C601AA27EE
:10BBF000BB275C016D01AE28BF28C02AD12AA2163E
:10BC0000B306C406D50660F525966CAD7DAD8EAD48
:10BC10009FAD2597615070408040904025966CAF55
:10BC20007DAF8EAF9FAF2597A20CB31CC41CD51C53
:10BC3000A214B304C404D50498F0A216B306C40633
:10BC4000D50670F4615070408040904025966CAFEE
:10BC50007DAF8EAF9FAF2597A20CB31CC41CD51C23
:10BC6000A21AB30AC40AD50AC601B501A4019301F8
:10BC70000E944C627B018C01C601B501A4019301B5
:10BC80000E944C62C901DA013C014D01C401B301BB
:10BC900021962CAD3DAD4EAD5FAD21970E940D625A
:10BCA0009B01AC018701FF24EE2489A59AA5ABA5D1
:10BCB000BCA5A070B07057016801A82AB92ACA2A89
:10BCC000DB2AA216B306C406D506E0F40894610880
:10BCD000710881089108A20CB31CC41CD51CA214C5
:10BCE000B304C404D50470F0A216B306C406D50686
:10BCF00048F408946108710881089108A20CB31CEB
:10BD0000C41CD51C8DA59EA5AFA5B8A96F960FAC78
:10BD10006F9704C0880F991FAA1FBB1F0A94D2F700
:10BD20008DA79EA7AFA7B8ABA21AB30AC40AD50ABB
:10BD30002596ECACFDAC0EAD1FAD2597D70199272C
:10BD40008827682A792A8A2A9B2A82012227332770
:10BD500029960CAF1DAF2EAF3FAF2997A2019101DD
:10BD6000407050702D962CAF3DAF4EAF5FAF2D970A
:10BD7000C601B50129962CAD3DAD4EAD5FAD2997FD
:10BD80000E944C627B018C01C601B50129962CAD45
:10BD90003DAD4EAD5FAD29970E944C62C901DA01FD
:10BDA00061968CAF9DAFAEAFBFAF6197BC01CD01C7
:10BDB0002D962CAD3DAD4EAD5FAD2D970E940D6221
:10BDC0009B01AC018701FF24EE24ADA4BEA4CFA447
:10BDD000D8A8C601AA27BB2757016801A82AB92AF3
:10BDE000CA2ADB2AA216B306C406D50660F56196F8
:10BDF0006CAD7DAD8EAD9FAD619761507040804060
:10BE0000904061966CAF7DAF8EAF9FAF6197A20CF3
:10BE1000B31CC41CD51CA214B304C404D50498F0EC
:10BE2000A216B306C406D50670F461507040804077
:10BE3000904061966CAF7DAF8EAF9FAF6197A20CC3
:10BE4000B31CC41CD51CA21AB30AC40AD50AC60165
:10BE5000B50129962CAD3DAD4EAD5FAD29970E9441
:10BE60004C627B018C01C601B50129962CAD3DAD1C
:10BE70004EAD5FAD29970E944C62C901DA015C01A9
:10BE80006D01C601B5012D962CAD3DAD4EAD5FAD3A
:10BE90002D970E940D629B01AC018701FF24EE24C7
:10BEA0008DA59EA5AFA5B8A9A070B070E82AF92A03
:10BEB0000A2B1B2BE216F30604071507C0F408949F
:10BEC000A108B108C108D108E20CF31C041D151D1E
:10BED000E214F3040405150550F0E216F306040716
:10BEE000150728F40894A108B108C108D108619683
:10BEF000ECACFDAC0EAD1FAD6197D701992788273B
:10BF000096018501082B192B2A2B3B2B09AB1AAB69
:10BF10002BAB3CAB62C26E147F048006910608F422
:10BF200051C220E0E21620E0F20621E0020720E004
:10BF3000120788F43FEFE316F1040105110531F013
:10BF400028F048E050E060E070E017C040E050E0CA
:10BF500060E070E012C040E0E41640E0F40640E02B
:10BF6000040741E0140728F048E150E060E070E089
:10BF700004C040E150E060E070E0D801C701042E49
:10BF800004C0B695A795979587950A94D2F78554DE
:10BF90009E4FDC012C9130E2A32EB12CC12CD12C70
:10BFA000D601C501841B950BA60BB70B821B91090B
:10BFB000A109B1090097A105B10589F4E614F704B8
:10BFC0000805190508F4F2C16DA47EA48FA498A8F1
:10BFD000621473048404950408F0E8C1F3C16E96FA
:10BFE0008FAF6E97082E04C0EE0CFF1C001F111FB0
:10BFF0000A94D2F76A2D681BD201C101062E04C033
:10C00000B695A795979587950A94D2F75C016D012F
:10C01000AE28BF28C02AD12AADA2BEA2CFA2D8A6E0
:10C02000720161016E960FAC6E9704C0CC0CDD1CE2
:10C03000EE1CFF1C0A94D2F7C9A2DAA2EBA2FCA262
:10C0400064015301062E04C0D694C794B794A794F4
:10C050000A94D2F7D401C3016E960FAC6E9704C058
:10C06000880F991FAA1FBB1F0A94D2F7EDA4FEA444
:10C070000FA518A904C016950795F794E7946A953B
:10C08000D2F737014801682A792A8A2A9B2A6D8EBD
:10C090007E8E8F8E98A2EDA0FEA00FA118A538016C
:10C0A00088249924980187012070307065960CAF20
:10C0B0001DAF2EAF3FAF6597C601B501A401930137
:10C0C0000E944C627B018C01C601B501A401930161
:10C0D0000E944C62C901DA011C012D01C201B101AB
:10C0E00065962CAD3DAD4EAD5FAD65970E940D627E
:10C0F0009B01AC018701FF24EE24AD8CBE8CCF8C5C
:10C10000D8A0C601AA27BB2757016801A82AB92AC7
:10C11000CA2ADB2AA216B306C406D50600F508947F
:10C120002108310841085108EDA0FEA00FA118A573
:10C13000AE0CBF1CC01ED11EAE14BF04C006D1067B
:10C1400070F0A216B306C406D50648F40894210878
:10C15000310841085108AE0CBF1CC01ED11EA21AE6
:10C16000B30AC40AD50AC601B501A40193010E940D
:10C170004C627B018C01C601B501A40193010E94B0
:10C180004C62C901DA013C014D01C401B30165965D
:10C190002CAD3DAD4EAD5FAD65970E940D629B012C
:10C1A000AC018701FF24EE248D8D9E8DAF8DB8A14B
:10C1B000A070B07057016801A82AB92ACA2ADB2AE0
:10C1C000A216B306C406D50600F5089461087108E6
:10C1D000810891086DA17EA18FA198A5A60EB71E1A
:10C1E000C81ED91EA616B706C806D90670F0A21634
:10C1F000B306C406D50648F408946108710881089E
:10C200009108A60EB71EC81ED91ED601C501821BF5
:10C21000930BA40BB50B898F9A8FAB8FBC8FD10179
:10C220009927882764015301A82AB92ACA2ADB2A38
:10C23000A9AABAAACBAADCAA860175012FEF3FEF03
:10C2400040E050E0E222F32204231523A6016627F2
:10C2500077276D964CAF5DAF6EAF7FAF6D97A9A09E
:10C26000BAA0CBA0DCA06FEF7FEF80E090E0A62229
:10C27000B722C822D92289A19AA1ABA1BCA11D01D4
:10C2800044245524C801B701A60195010E940D62FE
:10C2900069966CAF7DAF8EAF9FAF6997C801B7014C
:10C2A000A20191010E940D623B014C016D966CADA3
:10C2B0007DAD8EAD9FAD6D97A60195010E940D627B
:10C2C0007B018C016D966CAD7DAD8EAD9FAD6D9794
:10C2D000A20191010E940D625B016C01A80197010E
:10C2E000260D371D481D591D69966CAC7DAC8EAC72
:10C2F0009FAC6997C401AA27BB27280F391F4A1F83
:10C300005B1F2E153F054007510748F4E12CF12C27
:10C3100061E0062F112DAE0CBF1CC01ED11ECA013C
:10C32000AA27BB27BC01CD016A0D7B1D8C1D9D1D5D
:10C33000698C7A8C8B8C9C8C66167706880699069D
:10C3400040F1661577058805990509F043C0D901C4
:10C350009927882769962CAD3DAD4EAD5FAD6997A5
:10C3600040705070820F931FA41FB51F2DA53EA5CE
:10C370004FA558A96E960FAC6E9704C0220F331FBD
:10C38000441F551F0A94D2F7281739074A075B073D
:10C3900008F509A91AA92BA93CA901501040204071
:10C3A000304009AB1AAB2BAB3CAB14C066247724EE
:10C3B000430121E030E040E050E029AB3AAB4BAB29
:10C3C0005CAB0BC066247724430119AA1AAA1BAAE6
:10C3D0001CAA03C0662477244301FE01719688E0FD
:10C3E000DF011D928A95E9F7A9A8BAA8CBA8DCA815
:10C3F000A98ABA8ACB8ADC8A6D8A7E8A8F8A988ECD
:10C4000029A93A894B895C89662D7E898F89988D07
:10C41000C25ADF4FE2E10C94A562629FD001739F84
:10C42000F001829FE00DF11D649FE00DF11D929FD0
:10C43000F00D839FF00D749FF00D659FF00D99270F
:10C44000729FB00DE11DF91F639FB00DE11DF91F33
:10C45000BD01CF0111240895991B79E004C0991FF3
:10C46000961708F0961B881F7A95C9F7809508954E
:10C47000AA1BBB1B51E107C0AA1FBB1FA617B7070A
:10C4800010F0A61BB70B881F991F5A95A9F7809526
:10C490009095BC01CD010895A1E21A2EAA1BBB1BE9
:10C4A000FD010DC0AA1FBB1FEE1FFF1FA217B30780
:10C4B000E407F50720F0A21BB30BE40BF50B661F96
:10C4C000771F881F991F1A9469F76095709580955A
:10C4D00090959B01AC01BD01CF01089597FB092EFA
:10C4E00005260ED057FD04D0D7DF0AD0001C38F443
:10C4F00050954095309521953F4F4F4F5F4F089590
:10C50000F6F790958095709561957F4F8F4F9F4F6F
:10C5100008952F923F924F925F926F927F928F92E7
:10C520009F92AF92BF92CF92DF92EF92FF920F93C2
:10C530001F93CF93DF93CDB7DEB7CA1BDB0B0FB6CC
:10C54000F894DEBF0FBECDBF09942A883988488889
:10C550005F846E847D848C849B84AA84B984C8841F
:10C56000DF80EE80FD800C811B81AA81B981CE0F16
:10C57000D11D0FB6F894DEBF0FBECDBFED010895FB
:10C58000911106C080538A5010F0865C06C0089551
:10C5900099278827089585FDFBCF80629111F8CFF8
:10C5A00081568A51E0F708959111089581568A5174
:10C5B00008F4805285580895FB01DC010D9000209D
:10C5C000E9F7119705900D920020E1F70895FB011E
:10C5D000DC018D91059080190110D9F3990B089514
:10C5E000FB01DC0105900D920020E1F70895FC01AC
:10C5F00005900020E9F7809590958E0F9F1F089574
:10C60000FB01DC014150504030F08D9105908019C4
:10C6100019F40020B9F7881B990B0895FB01559177
:10C620005523A9F0BF01DC014D9145174111E1F7F8
:10C6300059F4CD010590002049F04D91401541116C
:10C64000C9F3FB014111EFCF81E090E0019708951C
:10C65000FB01DC0102C001900D9241505040D8F71F
:10C6600008956817790768F4FB01DC01E40FF51FF2
:10C67000A40FB51F02C002900E9241505040D8F74F
:10C6800008950C942863DC0101C06D934150504023
:10C69000E0F70895FB01DC010D900020E9F7119708
:10C6A00001900D920020E1F70895FC018191861719
:10C6B00021F08823D9F7992708953197CF0108955C
:10C6C000FB01DC018D91019080190110D9F3990BC8
:10C6D0000895FB01DC0101900D920020E1F708951F
:10C6E000FB01DC014150504030F08D9101908019E8
:10C6F00019F40020B9F7881B990B0895FB01DC01A0
:10C700004150504048F001900D920020C9F701C0FF
:10C710001D9241505040E0F70895DC01CB01FC012F
:10C72000F999FECF06C0F2BDE1BDF89A319600B48A
:10C730000D9241505040B8F70895A6E1B0E044E0B2
:10C7400050E00C948F63A8E1B0E042E050E00C941C
:10C750008F63DC01A40FB51F4150504048F0CB015E
:10C76000840F951F2E910E94BA6341505040D0F71C
:10C770000895262FF999FECF92BD81BDF89A0197B1
:10C7800000B4021639F01FBA20BD0FB6F894FA9A19
:10C79000F99A0FBE08950396272F0E94BA630E944C
:10C7A000B963252F0E94BA63242F0C94BA630196B3
:10C7B000272F0E94BA630C94B963DC01CB0103C03C
:10C7C0002D910E94E86341505040D0F70895262FE4
:10C7D000F999FECF1FBA92BD81BD20BD0FB6F89466
:10C7E000FA9AF99A0FBE01960895242F0E94E863E1
:10C7F000252F0E94E8630C94FD630E94E763272FB6
:08C800000C94E863F894FFCFEB
:10C80800020000000000C010000000000900010044
:10C8180000004600000000000000060100000000C3
:10C8280000090001000000460000000000000000B0
:10C8380000000000000100000046000000000000A9
:10C848000000000000090001000000460000000090
:10C858000000000000000009000100000046000080
:10C868000000000000000000000900010000004670
:10C8780000000000000000907E0000C8040215CDF2
:10C888005B07E5559A15B53B121F33134905F406A6
:10C89800140734075407504D544B0043593D59373A
:10C8A80059315949592B59A5583558CC57895546A6
:10C8B800555D57F156AE566B56DE55000102020320
:10C8C800030303040404040404040405050505051E
:10C8D80005050505050505050505050606060606FB
:10C8E80006060606060606060606060606060606E0
:10C8F80006060606060606060606060707070707CB
:10C9080007070707070707070707070707070707AF
:10C91800070707070707070707070707070707079F
:10C92800070707070707070707070707070707078F
:10C93800070707070707070707070708080808087A
:10C94800080808080808080808080808080808085F
:10C95800080808080808080808080808080808084F
:10C96800080808080808080808080808080808083F
:10C97800080808080808080808080808080808082F
:10C98800080808080808080808080808080808081F
:10C99800080808080808080808080808080808080F
:10C9A80008080808080808080808080808080808FF
:0CC9B8000808080808080808080808001B
:00000001FF
